:020000040000fa
:08000000020c040000000000e6
:020000040000fa
:10180000050000006f0b21000e7f24000e018800f0
:10181000000000000c000700404c260001002000e2
:1018200011000700000020000000e000020032006c
:101830000000020000000000a0680200000000009c
:101840000040da000000fe004440a90080f32000c0
:101850000000e0000300320000002000a00188002a
:101860004440a80000000600910188008000780034
:101870000000eb0015003700e280400032a0b40009
:101880009101ba00e280400032a0b4009102ba0097
:10189000e280400032a0b4000002eb00472bde00e3
:1018a000f507b200602ce10004003a000059eb009b
:1018b0008301e900fdff3e00040037006128e100dc
:1018c000010032000082eb00040007001101ba00a1
:1018d0000200e000e8ff3a00000006003159ba00bb
:1018e0008301e9000c0032002159ba008301e900ac
:1018f000080032000400e00003003a00e2804000eb
:1019000032a0b400f5ff370011d9ba008301e90015
:10191000faff3a008100e800e180400032a0b40004
:10192000000006000a00fa0080017800e20f500073
:1019300028003e00a0858000e10f50000800320022
:10194000802320000000e000050032000423200076
:101950002523200046232000800178000400370062
:10196000042220002522200046222000832220007d
:10197000144090000004e000040035008009eb00f2
:10198000144090000074a000104298001540900090
:101990000028a30003003a00154090000024a00096
:1019a000904298008001eb0007003700154090003e
:1019b0000008a300fdff320063c078000000fb00b8
:1019c000000b78008301e800828f5100f7ff3a0096
:1019d0000800370030002000b0bf9f00c3bf9f0049
:1019e000d1bf9f00e2bf9f006a80570000c0da00ad
:1019f0006fb99700020078000080fa00000006002e
:101a0000889fbe008a9fbe00010578000100e000ab
:101a10000400350008003c000000e0002000320017
:101a20000500370060001000e080180002003b0055
:101a300001f02c001a0037000004be006011b8004d
:101a40006b0920000982cf00020039000882cf0014
:101a50000441b000694252000e00320008003b0011
:101a600082817100610164008904d1000884d3007f
:101a70008b05e8000442e800f9ff3a000500370052
:101a80000804440089844c008b05e9000442e90005
:101a9000fbff3a002b0207000af0a70001f0a000ac
:101aa0004f05be004f04be000000060003f0a20078
:101ab000889fbe008a9fbe008c1f780047020700e7
:101ac0004e0233006450e1004f0032006420e10018
:101ad0005200320003826c0007003b000905d00071
:101ae0000306d000820f54000c065d00020039008e
:101af00002003200890178000306780085825500d3
:101b000004003d000003fd008103fd008502ea00a2
:101b10008b854200840f720002003b0060001000c1
:101b2000e08018006011b8000005eb007a28e100a1
:101b30000a00390006007800c75ddd00f707b20033
:101b4000878075002d003700828171000a017800be
:101b5000610560008180d1000080d3008502e9002a
:101b6000f9ff3b00060440008784480002003b0068
:101b700060041400e0841c000988a3000700320000
:101b80008a81710082817100610164008904d10041
:101b90000884d3008b05e800170037000978a300fc
:101ba00013003a000b00e000130034008b05e9003d
:101bb0000804440089844c000a4474000978a30096
:101bc0000d003a000b00e000070034008b05e9002f
:101bd0000804440089844c0001003a000b002000f6
:101be0000978a300f7ff32000001eb000200370084
:101bf000828171000a017800d20107000cf0a70071
:101c000001f0a000060237006420e10002003a0063
:101c1000838f6c00060233000801be000200be0084
:101c2000ff013700f4ff2f000402370014002000ea
:101c3000020237000001be001b0207000470a7006b
:101c400003f0a1006509b100160032000d00350057
:101c50006828e10006003500f0ff2f00f1ff2700a3
:101c60000300e00013003b00010028000000050015
:101c700000004000818048008502e900fcff3a0036
:101c800008003700f88f420002003c008000eb00a3
:101c9000000005008100d1000080d3008502e8002b
:101ca000fcff3a000300e00002003b00600010006f
:101cb000e0801800000006000001be00fa010700e5
:101cc0000470a70003f0a10003f8a30013003a007a
:101cd0006509b10010003200090035006928e100f3
:101ce000020035000100280000000500000040004f
:101cf000818048008502e900fcff3a0000000600f0
:101d0000f88f4200050035008100d1000080d3002b
:101d10008502e800fcff3a00000006008000eb00ae
:101d200000000500889fbe008a9fbe008c1f7800bf
:101d3000aa010700b101330003866c006450e10082
:101d40002e0032006420e100330032006150e100d7
:101d50002f0032006120e1003100320085855500fe
:101d6000eb07b00009002000080420000500370040
:101d70000804440089844c000a0031000603430033
:101d800087834b000001530081815b00f8ff330023
:101d90000203be000800a0000804440089844c002f
:101da000f6ff3900c639dd008301730001003200ff
:101db000130020008904d1000884d3000998a300ef
:101dc000050032000800a7000300a0008904d1002c
:101dd0000884d3008b05e8008904d1000884d3006f
:101de0000001eb000281d2005601070001f0a100c2
:101df0000cf0a70001f0a000890137006420e10089
:101e00008b0132000801be000200be00f7ff370060
:101e10006120e100860132006000b800f3ff370066
:101e20000000200001f82700f0ff3700889fbe0067
:101e30008a9fbe008c1f7800680107006f01330085
:101e400003866c006450e100240032006420e1004d
:101e5000270032006150e100220032006120e100e1
:101e6000210032008b854200eb07b1000134b8003d
:101e7000003ab8000804420089844a00013ab800d8
:101e80000030b8008880400009014a000400330097
:101e90000000400081804800020149008b05e900f4
:101ea000c909dd0083017000010032001300200029
:101eb000c814de004814dd004709de001200b2003d
:101ec000c808de00088470001e01070001f0a100b0
:101ed0000cf0a70001f0a000510137006120e100e3
:101ee000530132000801be000200be00f7ff3700b8
:101ef0006150e100fcff3a004d0137000c00fa0090
:101f0000889fbe008a9fbe008c9fbe0033010700e1
:101f10000206be00840578000200be000200200018
:101f20007601070005003a008b02b3001200200082
:101f30007201070001003a00f8856d000c01be0037
:101f4000c60007000800be009b0032000b08a3007b
:101f50009e003a000df0a7000be0a00009f0a700da
:101f60000bf0a00009f0a1000801be00bb000700b3
:101f70000bf0a6009500320001003c000bd0a00041
:101f80008acf7500b20033006000b8006250e100f3
:101f900099003900a1003e000b28a300a2003a00de
:101fa0000bf8a300060032000b58a300a700320074
:101fb0000801be00a90007000800be00940032001e
:101fc0000800be00740107000004be00050578008b
:101fd0000bf0a7000b30a6000bf0a1005b079800e8
:101fe000324f200053f3230010ff070005003d008f
:101ff0000800be0012002000740107000004be00ab
:102000000a05e9004a0798006150b9007cfe070004
:10201000008fbe000c01be0084ff070005ff070013
:10202000300798000100e00002003d006000100051
:10203000e0801800f2ff2700820f5000e08f580068
:1020400064003e000c00be00fafe07002007980066
:10205000f2072000820f5000e08f580005003c007e
:1020600012f82f00f3ff2f00820f5000838f5800cb
:1020700009003d000a00e0000300320001003c00be
:102080000201ea00020578006000b800200798000d
:102090003a079800190037003e0090006100b9002f
:1020a00057fe0700809fbe000c00be004109dd0006
:1020b0004811de007208b100100107000005be00e3
:1020c0001e01be0059ff07004f01be0077fe07004a
:1020d000809fbe000c00be000a01be0073fe070018
:1020e0001e01be0051ff07004f01be0070fe070039
:1020f0008221270013f323004cff07000005be00d8
:102100002e0090006100b9003dfe070001f0a20022
:102110000c01be0066fe07000006be000800be00ff
:102120004c0107000c01be0040ff07000a01be0081
:102130005ffe0700809fbe004a0007002e0590004a
:102140000af0a7000a05ea00050037000800be00f3
:102150000801be0035ff07000004be000c00be00f1
:102160000801be000a00a70030ff07000006be00fd
:102170000a05d100f5ff3a005e01900002e0a600da
:10218000030037000001be0036000700e5fe07002f
:102190000004be004f00be00850107000801be001c
:1021a00022ff07003e01900008010700de059000b5
:1021b0000bf0a70001f0a2004f06be004f05be00c5
:1021c0004f04be000080fa00000006002500070052
:1021d000f9ff3700270007006000b8000bd0a70008
:1021e0000bc0a0000be0a7000bc0a2000bc0a70013
:1021f00001f82700f0ff37000df8a30002003200bd
:102200001e000700190007000bf8a300eaff3200c8
:102210000b30a70001f0a200e7ff37000df8a30084
:10222000f9ff3a00f7ff37000801be000b00070076
:10223000e6ff320001003c000df0a2006000b80093
:102240000df0a70009000700dbff37000b000700b7
:10225000f1ff2700f0ff2f00d7ff37000100070034
:1022600072fe370001f823000000050001f8270086
:1022700000000500200220000100370010022000ad
:10228000e072880000000600809fbe00821f780078
:102290000001eb0099000700cf027800808abe00a1
:1022a0000001be004f00be0000fe3a000470a60010
:1022b0006000b80003f0a70001f0a00000000600d5
:1022c000040020005d0037006022b80006022000f4
:1022d0000000d0008180d2000482d2008582d2002a
:1022e0000000a0000202520083825a000300310065
:1022f0000202420083824a000000a1000603e900b6
:10230000f3ff3a0000000600839f68000100e00030
:1023100002003d0060001000e08018000300e000b3
:1023200002003d0060011100e0811900e6ff070096
:102330004f00e00002003b0060001000e080180049
:102340000000060081002000618055000b003d0068
:102350000b00200061fe2f000100e1001d00340091
:1023600082817100610164008904d1000884d30076
:102370000000e800faff3a007100200061006400ec
:102380000300700002006000090032006104440094
:10239000e0844c000988a500050032008b05e800a8
:1023a0006808e10002003a008904d1000884d300e3
:1023b000f20f20000258e10005003d00c75ddd007e
:1023c000f907b20089807500080078000000060057
:1023d0000bf827008b007800000005000004be0009
:1023e000310007000003be000405be000200be006d
:1023f0002d000700844f7500000006000200be009b
:102400006450e100050036006420e100020036005f
:102410000968a30001003a000800be000160a000a6
:102420004f0678004f05be004f04be0000000600b6
:10243000f0ff2f00f1ff2700f9ff3700889fbe0053
:102440008a9fbe00841f7800e4ff07004f007800d9
:1024500011003300f0ff2f00838f6c0006003b005b
:10246000040565000a00a7000800370009f0a6006f
:102470001000200008003700820f5400838f5c009a
:10248000030039001000200001003e000000200081
:1024900009f0a7000000ea004f05be004f04be008f
:1024a0000000e00000000600c70ade00f107b200ed
:1024b000f50fb20008003200e1cf42000200320006
:1024c0000170a00024000500810f7000010032009f
:1024d0000408050044000500810f700002003a0066
:1024e000140005008502e9000000400081c048009a
:1024f000fcff3b000170a00024000500889fbe0087
:102500008a9fbe000003be00e7ff07008505780034
:1025100082815200020020006220e10004003a00a3
:10252000f307b100040035007718e100040035001e
:102530000600be00140037006000b8000f0037002e
:10254000f50f2000faff2f008502d1000a85d30085
:102550008301e900fcff3b00818462000004650008
:10256000890f7400f2ff32008582ea000a85ea00d2
:10257000818462000004650072ff070007f0a70075
:1025800001f0a0000081eb000200e0004f05be005a
:102590004f04be00000006000003be00c2ff07009b
:1025a0006220e100020032000600be0005000500c6
:1025b000e507b100f107b20004f023008480700049
:1025c00007f0a70001f0a000240005000003be00f2
:1025d000b5ff07006220e100020032000600be00e5
:1025e0000000060085024100e30f20000328e100ff
:1025f00005003c00a3fe2f000328e10007003d007a
:102600000500200001003700f50f20002002200007
:10261000e07288006000b800080037001300200056
:102620008381520005003d008100d1000080d3006d
:102630008301e800fcff3a0005002000c72add0006
:10264000f107b2008580700007f0a70001f0a0003c
:1026500000000600889fbe008a9fbe008c9fbe00bf
:10266000cdff0700850478000005be006420e1006e
:1026700049003e006220e1000300320009003500fd
:102680000bf8a300440032000bf8a300080032004e
:1026900010022000e0728800f0ff2f00f1ff2700f9
:1026a0003d00370001f82f00000020003a003700fd
:1026b0003d000700fdfc07000006be000a00be004a
:1026c000324f200053f3230056fd0700060034006c
:1026d0000c00be0034000700f4fc07000006be003a
:1026e0000a00be00020037008904e9000c00be00a9
:1026f0002d000700cdfd07002b000700ecfc0700b4
:102700000001be000c00be0086fd07000005be00f3
:102710000001be00c5fd07000006be00a2f32300b5
:10272000430d2c00e2fc0700809fbe000c00be00a1
:10273000d2e32700d3f02b00bcfd07004f01be0001
:1027400078fd07000006be000a01be00b7fd0700c5
:102750000a01be00d6fc07000006be006148b900b1
:10276000a7fc07000005be0032082800e3952b00f7
:10277000aefd07000c01be00cdfc07000006be0048
:102780000a00be000200280013f32300a7fd070083
:102790000c01be00c6fc07004f06be004f05be0080
:1027a0004f04be000000060003f0230002000500f5
:1027b000889fbe008a9fbe008c9fbe000004be00a2
:1027c00039ff07000800be006420e10048003e0019
:1027d0005500320072212700132b240011fd070041
:1027e00047003c000800be00c2ec2800e32c2c008f
:1027f0000efd0700470035000800be0001f0a100f3
:10280000020020000338230008fd070043003500c4
:102810000800be00b2a32a0083fb230083fd07004b
:102820000200200003f0230001f0a70003f0a00045
:102830009ffc0700fffc07000005be0070fc0700be
:1028400001f0a2000006be000200280013f32300de
:1028500076fd07000801be0095fc0700809fbe00c2
:102860000c00be0032082800e3952b006ffd070026
:102870004f01be008efc07000006be000001be0036
:102880006afd0700809fbe004241250083b82300f7
:1028900066fd07000200200003e8230084fc070017
:1028a0000c01be0061fd07000006be004f00be0027
:1028b000f2f92b00c3d423005cfd070002002000c6
:1028c00003f023007afc07000c01be0077fc070030
:1028d0000001be000c00be0012fd07000200200037
:1028e00003f0230072fc07006101450037ff070079
:1028f0004f06be004f05be004f04be00000006009c
:1029000001f827000000200022022000e272880067
:10291000f7ff37006000b800fbff370001f8230025
:1029200000002000f2ff370009f8a300f0ff32009a
:102930006000b800eeff3700881f780000047800c0
:102940005001be004000be000400400085804800e9
:102950000601490087814900009cbe000294be0028
:102960000400e1000588e1000690e1000798e1001d
:1029700002003100680044001008e8004f047800ad
:1029800000000600f4874700889fbe008a9fbe00b3
:102990008c9fbe008e1f78000205be000004be00a2
:1029a000d4b79f00e5b79f00f6b79f0087bf9f0091
:1029b0000000eb00c0b79f00b0b79f00a0b79f001a
:1029c00090b79f0080b79f000d042000bfb0970014
:1029d0004fb09700000140000000e0000f003d00f4
:1029e0004f08de0000007100c0b79f009e00070086
:1029f00001003d0012002000a100070001003d0081
:102a000012002000a6000700b1000700b600070072
:102a10000f004000c8ff0700220037004f08de000b
:102a200000067100ccb79f008f00070001003d0039
:102a3000120020009200070001003d00120020005b
:102a400097000700a20007000fb297009fb29700ff
:102a50002fb39700bfb39700a900070000005200f2
:102a600081805a0002015b0083815b0080b79f0078
:102a700091b79f00a2b79f00b3b79f000007eb007c
:102a80009f0007000020e10001a8e10002b0e10082
:102a900003b8e100010031001e0020000e005600c6
:102aa000c0b79f004fb297000400e0000700350058
:102ab00010002000010020006011b8000804700020
:102ac000898470000a0571008b8571008d06e9000c
:102ad000beff3a000400e00003003d008200070052
:102ae0000f00400094ff07004fa897000000e0008f
:102af00004003a000fb497009fb497002fb59700d9
:102b0000bfb59700940007004f0778004f06be003e
:102b10004f05be004f04be004f01b100000006008b
:102b2000881f780018002000881f780095ff070094
:102b30008f87e9004f04780000000600801feb003b
:102b400090ff07008f87e90000000600889fbe0005
:102b50008a9fbe008c1f78006e00070007003d00b2
:102b600073000700e00f5b00e08f5b0007003d0093
:102b7000320007000006eb000400370034000700b5
:102b800002003d002a0007001c0020007200070020
:102b9000e3ff07000203be000002be000c00e000dd
:102ba00001003200220007000400be000601be0042
:102bb0004f0678004f05be004f04be00000006001f
:102bc000889fbe008a9fbe008c1f780051000700be
:102bd00005003d0056000700e00f5b00e08f5b0042
:102be00006003d00040037001900070003003d0007
:102bf0006000b8006011b800100007005600070020
:102c0000ceff07000203be000002be000c00e00081
:102c100001003200060007000400be000601be00ed
:102c20004f0678004f05be004f04be0000000600ae
:102c30006000b8006011b8000000370004025000c6
:102c4000858258000603590087835900000006005a
:102c50000006eb00e00f5200e08f5a00e00f5b002f
:102c6000e08f5b00000006000180400090b79f00ed
:102c70000001eb008fb097000100e00000000600ab
:102c80000200700090b79f000180400080b79f0055
:102c90000001eb00ffa897000100e0000000060023
:102ca0000200700080b79f00018040006faa97006b
:102cb000cf20de0001007000f0af9f000402420050
:102cc000250007004f18de00000272000000060019
:102cd000e4af9f000804440089844c000a054d00bd
:102ce0008b854d00000006003fb29700cfb29700e1
:102cf0005fb39700efb3970000fe2f0000000600bf
:102d00003fb09700cfb097005fb19700efb1970049
:102d1000000006000205be000004be00e00f5000e7
:102d2000e08f5800e00f5900e08f590000000600c6
:102d30006000b8006011b800080450008984580091
:102d40000a0559008b8559001c002000e00f520035
:102d5000e08f5a00000006000800be000a01be0015
:102d6000000006002800fa00889fbe008a9fbe006f
:102d70008c9fbe0003866b000c0207000028a30096
:102d800064003a000128a30067003a000008a3008d
:102d900062003a000108a30065003a001e0090009e
:102da000be08900081064000ed3fb100f48057005e
:102db000ee019000111ab8008e099000311bb80086
:102dc0009e099000311cb800511db800f4855700d1
:102dd00046000700fe0190003a0007008b85e800de
:102de0003e0007008e09900040000700ee019000b1
:102df000340007008b85e800380007008e0990003a
:102e0000400007009e0990001b18b800890440008c
:102e10000a854800fe019000340007008b85e80019
:102e200038000700ee019000300007008e09900086
:102e30001b18b800890440000a8548000a98a300be
:102e400008003a000402420085824a0006034b0053
:102e500087834b0008044c0089844c000a054d0010
:102e60008d06e90084827200850273004c3add0011
:102e7000850272000100320015002000443ade0095
:102e80001400b2004538de00cb45dd000b007000b9
:102e9000c540de00cb4ddd008b8070004549de0073
:102ea000cb55dd000b017100c551de000d0378002c
:102eb000d701070003f0a1000cf0a70003f0a00069
:102ec000ce0137001b18b800850240000683480079
:102ed000e0834b0060044c00070037001b18b8006b
:102ee0000603400087834800faff37001b18b8002c
:102ef0008703400008844800e0844c0060054d00d2
:102f0000000006001b18b80008044000898448002f
:102f1000faff37000108a300b5013a005800be00cf
:102f20005801be00e3ff37000008a300b0013a00db
:102f300009047800f9ff3700810378005afd070083
:102f40000001be006000b8000478a30013003a003e
:102f50006220e10015003e000d0039008301d10020
:102f60000281d3008180d3008301d1000281d3008c
:102f70008180d3008301d1000281d3008180d300fe
:102f80000538b000c42add00f300b200838172006e
:102f900007f0a70003f0a00000000600f3ff2700e1
:102fa000f2ff2f006110b900fbff370003ff27007d
:102fb000f7ff37008f1fd100c10107008f87e9009d
:102fc0000000e00000000600801feb00bc010700cd
:102fd0008f87e9000000e000000006001400fa00fe
:102fe000889fbe008a9fbe008c9fbe000005be0069
:102ff0000206be00680047000c90be000a90be00aa
:10300000d80107006400e1001a00320016003e00fb
:103010006100e1001a0032006e049000fe0490008e
:103020000e0b90009e0b90006011b8009e05900062
:103030000b38b100d501200082817100610164006c
:103040008703d1000683d3008984d3000884d3008a
:103050008502e900f8ff3a00bafc07000df0a7006e
:1030600001f0a00065013700f1ff2700f0ff2f00fd
:103070006201370001f8270000002000f7ff370049
:103080006000b800f5ff370043fd07000509780030
:1030900000000600809feb00890107008f87e90090
:1030a0000000e000000006002800fa00889fbe0033
:1030b0008a9fbe008c9fbe00070678008786690045
:1030c0000c003b00030478008704780008f0a1009e
:1030d00009f0a100840f5000858f5800860f590019
:1030e000890f5c00030033000cf0a20001003a00dd
:1030f0000cf0a1002d0107006400e1005f00320028
:10310000780147006408e100610032006c0147006b
:10311000748557003200be001201be003a04be00a2
:103120001a05be001e039000be0a900085035300de
:1031300006003d000004fd008104fd000205fd00c5
:103140008305fd008703ea00050378000df8a3005e
:103150000400320060041400e0841c0060051d00bf
:10316000e0851d006022b8007d0320000d38e100dd
:103170008006eb000b0039004433dd00f300b200a1
:103180008301730039003700848272000d027800d9
:10319000e10664008b85d1000a85d3008984d300c1
:1031a0000884d3008703e900f7ff3b0008004000d4
:1031b000898048000a0149008b81490004003b00d6
:1031c00060001000e080180060011900e081190023
:1031d0000358a300090032008d82720084827200bd
:1031e000610260008301d1000281d3008180d3009d
:1031f0000080d3000603e8001b0037000348a3004b
:1032000017003a000600e000170034000603e9004a
:103210000d00a30000004800818048000201490021
:10322000838149000348a3000f003a000600e00034
:10323000090034000603e9000000400081804800d6
:10324000020149008381490001003a000003eb00bc
:103250000348a300f5ff32006022b80002003700e7
:103260008482720061826600e900070003f0a10019
:103270000cf0a70003f0a000e00037006401470055
:103280006408e10002003a000df8a300d8003a00fb
:103290003200be001201be00d80037001400fa0050
:1032a000889fbe008a9fbe008c9fbe000004be00a7
:1032b0000205be00680047000a90be000890be00ec
:1032c000280107000070a7000bf0a1000bf8a30075
:1032d00020003a009e0990000e099000fe00900028
:1032e0006e0090009e0290003443200084825200c1
:1032f000c20032000a003c00b4fc2f000428e100a8
:10330000140034008301d1000281d3008180d300f6
:103310000080d3008502e800faff3a00b7003700ca
:10332000b40020000428e10007003c000000400039
:103330008180480002014900838149008502e9003b
:10334000faff3a00ad003700030028000200200019
:10335000010037006011b8006000b800a700370016
:103360002800fa00889fbe008a9fbe008c9fbe0086
:1033700003866b008d0007006400e100440032000a
:103380006408e1004a0032006100e10046003200ba
:103390006108e10049003200ec0647006000b80017
:1033a0003d02be003d03be00f48657006011b80028
:1033b0003d04be003d05be007d0320000b0037002c
:1033c0000000a0008d06e900130032000402420054
:1033d00085824a0006034b0087834b0000004000b3
:1033e000818048000201490083814900080252009f
:1033f00089825a000a035b008b835b00f0ff3b006d
:103400000802420089824a000a034b008b834b006a
:103410008d06e900edff3a00848272008682720018
:10342000f707b20087827200010032001500200009
:103430001e0490003e0b900006035400e63fb000cf
:103440000368a300070032000000a7000500a000e9
:103450008301d1000281d3008180d3000080d3009a
:103460000603e8008301d1000281d3008180d300ec
:103470000080d3000002eb000482d2006400070049
:1034800003f0a1000cf0a70003f0a0005b003700e0
:10349000640247006408e100550032003400be00b9
:1034a0003401be00f6ff37006108e1005000320031
:1034b0006011b8006000b800f1ff370003ff27007b
:1034c00002002000fbff3700889fbe0083047800c5
:1034d0000300e0002c00350003003c000082700077
:1034e000040271002600320036432000c50020008f
:1034f0008383cf000a0039000541b1008283cf00e9
:10350000070039000541b1008183cf000400390074
:103510000541b1008083cf00010039000541b100b1
:1035200085c353006022b800120032000a003b003d
:1035300084827200610260008301d1000281d300a5
:103540008180d3000080d3000603e8008743e800b1
:10355000f7ff3a0007003700000040008180480074
:1035600002014900838149000603e9008743e9001d
:10357000f9ff3a002600070009f0a70003f0a000b9
:103580004f04be000000060060001000e08018003c
:1035900060011900e0811900d3ff3b00033e2c00bd
:1035a000f7ff370007f0a200bffe370068044700ae
:1035b0000294be000094be00fc0447008694be0046
:1035c0008494be00090078006600070008007800b7
:1035d0006400070099007800814f70000b003b00e9
:1035e0000800be00860007004f00b100030037004e
:1035f000f3ff2700f2ff2f006110b9004f06be0055
:103600004f05be004f04be000080fa000000060017
:103610001800200057002000080453000d003d0052
:103620000600200097fc2f000740e1001e00340038
:1036300084827200610260008301d1000281d300a4
:103640008180d3000080d3000804e800f8ff3a002e
:103650004700200061046000050474000404640055
:103660000d00320061004000e08048006001490028
:10367000e081490003b8a500070032000603e80016
:103680006538e10004003a008301d1000281d300d3
:103690008180d3000080d300f87f20000830e10053
:1036a00003003500080378006000b8006011b8001e
:1036b0004433dd00f300b200830173000000060014
:1036c000889fbe008a9fbe008c9fbe000404be007f
:1036d0000605be00809fbe00829fbe005600070008
:1036e000040678000800be000a01be005200070070
:1036f000840678004f03be004f02be008d4f760057
:103700007fb0970013003300f0ff2f008b8f6b000a
:1037100006003b000d0666000c00a7000a003700fb
:1037200007f0a600100020000a003700880f5200a2
:10373000898f5a008a0f5b008b8f5b000300390072
:103740001000200001003e000000200007f0a7004c
:103750000000ea004f06be004f05be004f04be0049
:1037600000000600800078005002be005003be003a
:103770004439de00f700b200f37f2000030161004e
:10378000090032000218e10016003a0085017200bb
:1037900083017300838173000008200015003a0044
:1037a0004000200013003700850172008301730080
:1037b0008381730005003a0004a8be0006a8be007d
:1037c000100020000b0037000201e9000402420053
:1037d00085824a0006034b0087834b000748a300fd
:1037e000f9ff32000740a00004a8be0006a8be00f2
:1037f0002000200080009800920098000000060041
:10380000e48240001078a300070032006402400008
:103810001178a3003400be001401be000400320081
:103820000330a700000006003500be001501be00f1
:103830000330a0000000060005ff2700058261009c
:10384000070032000428e1000100320024000500d6
:103850000600070001003a004400050004080500c6
:1038600002000700f9ff3a00140005006f826100b2
:10387000810270008502710085027200000006005e
:103880000c00fa00889fbe0000047800cfb09700bb
:10389000f0ff2700d0bf9f008004eb0099bf9f007e
:1038a00088bf9f00a8bf9f00200c2000b0bf9f00d2
:1038b00078815700708057005f0007000fb89700ad
:1038c000094878000fb897000804500008007800f5
:1038d0004f04be000080fa0000000600889fbe0072
:1038e0008a1f7800804078000004e00021003d003d
:1038f0008040ea00d0c6b30080cf500009003400f9
:103900008104fb0042062000110009008204d80057
:1039100000017800010078004311dd00eae5200095
:103920001f0037000100fb00e3e5200039003700ed
:10393000a2002000110009000200d8000001780058
:10394000010078004311dd00030141004300dd0068
:10395000030040003002be002003be004220900061
:10396000d2209000f221900062219000fdfc07001f
:103970002e003700d0c6b30080cf500023003400a3
:103980008104fb0042062000110009008204d800d7
:1039900000017800010078004311dd00eaf020000a
:1039a0000a014100a8002000110009000800d80009
:1039b0004300dd000a00400040229000d022900029
:1039c00060239000f023900002889000928890007d
:1039d000b289900022899000e2fc0700801f7800e5
:1039e00001027800110009008804d8000102fd00de
:1039f0004f0078000402fb004322dd000a0242006f
:103a00005403be004402be00d8ff37000100fb0093
:103a1000e3f02000eacf5000c5ff3c004300dd008a
:103a2000030040005001be004000be004f0578007a
:103a30004f04be00000006008f03b000889fbe0048
:103a40008a9fbe008c9fbe008e1f7800e0b79f004b
:103a5000f1b79f0082bf9f000000eb00a0b79f005e
:103a6000e60437008001eb0050c2b30080cf500065
:103a7000090032000100fb00efb09700ec040700e2
:103a8000e10f4000dd043200afb097008100e80094
:103a9000a1b79f00d90437007fb19700924078000a
:103aa000d0c2b30080cf50000c00320007003c00b1
:103ab0006d40500080cf50000d0032006b40400040
:103ac00080cf500019003a000e00370000c3b30049
:103ad00080cf500015003a000f0037000330a000df
:103ae0007fb297000402e800f4b79f00eaff3700b6
:103af0000300a000ffb297008502e800f5b79f0021
:103b0000e5ff37000310a0007fb697000c06e80021
:103b1000fcb79f00e0ff37000320a0007fb09700b4
:103b20000000e800f0b79f00dbff37000318a30098
:103b3000010032000300a1000338a300010032009d
:103b40000320a1000100fb0002fd2f000200400045
:103b5000e90f500010003e008000eb00c1b79f004d
:103b6000020278004fb197006a10b900ffb29700c7
:103b70001501fb000001410004014100c2b79f0094
:103b80005500fb00f5b79f0004004000e90f50000e
:103b90000d003e00f3ff37000006eb00ccb79f009e
:103ba000a0c2b30080cf500007003a000fb89700c2
:103bb000c000780080bf9f00c1b79f007fb1970011
:103bc0000201e800f2b79f00e0c2b3007fb29700a5
:103bd000944f100021003a00830678000de0a00009
:103be0008400e80064405000914f1000040032004f
:103bf000f1b79f008002eb00b5b79f0010003700bf
:103c00000fbe97004c0078008cbf9f00b0b79f009c
:103c1000ffb097008180e800f1b79f0013003700e4
:103c20003fb297006a20b900000041000300400045
:103c3000b0b79f00ffb297008502e800f5b79f007c
:103c40007fb697001c01fb0003fd2f00030041001d
:103c5000e90f5000f2ff36000400370083067800b9
:103c60000dc0a0000000eb00b0b79f007fb197002f
:103c7000b2407800f2b79f00c17f9f00c0c6b3007a
:103c800080cf50002700320014003c0068405000f4
:103c900080cf50009d00320009003c006c40500075
:103ca00080cf5000290032006b40400080cf500090
:103cb000720032000104e000560432008e0037002a
:103cc00060c6b30080cf50001c003200634040004b
:103cd00080cf500088003a008c00370030c7b30016
:103ce00080cf50001c00320007003c0064405000b0
:103cf00080cf5000130032000040e80080cf500019
:103d00007d003a001100370050c7b30080cf50004b
:103d10007d0032006340400080cf500076003a00c2
:103d20000b003700000028000d48a30001003a00f6
:103d30000001200080867600ccff37000da0a00097
:103d4000720037000d60a000700037000d50a00019
:103d50000d70a0006d0037008fb997004300780008
:103d600083bf9f00000478000000e00001003a00db
:103d7000e80521008004eb00010037008104e80021
:103d800089007800088044001004e000fbff3a003e
:103d90003fb297000400e00003003200890f520098
:103da00001003100840478000007eb00cfb29700d7
:103db000898f520001003600098752004368de00f7
:103dc000e106600019003a000d067800090037008e
:103dd000efb097000002200015040700e10f40003b
:103de000030032002fb097000000e800a0b79f004a
:103df0000c06e8008e0f5600f5ff3a000087eb0036
:103e00000a003700880078003100fb0001047800c8
:103e1000efb0970006040700e10f400003003200f6
:103e2000afb097008100e800a1b79f000900e9004a
:103e300080047800e10f4000f2ff3a000006eb003a
:103e40000d00e0000a003a00ec033700efb09700e5
:103e500000022000f6030700e10f400003003200db
:103e60002fb197000201e800a2b79f000c06e800fe
:103e70008e0f5600f5ff3a00e00337008fb9970028
:103e80004300780083bf9f00cf80de0001017800ef
:103e9000820178000205be000004be000203be00dd
:103ea0000002be004822de00482edd00040276003b
:103eb000c47f9f000d48a3000a0032000404e00004
:103ec00008003200e14f420006003200d1fb2f0013
:103ed000018047000448780018409800290020001d
:103ee00002003700d07f9f0019002000d2fb2f0076
:103ef00002844700a6ff3700c3fb2f00038447005e
:103f000019002000a2ff37000d0cb3000070200044
:103f100000826600270232000dc8a30002003200b2
:103f200064002000b4b79f000d48a30005003200d4
:103f30000fba97004401be004400be0084bf9f003a
:103f4000040037008fba97004500be0085bf9f0070
:103f5000f9fb0700e0af9f00f1af9f0082b79f0021
:103f600093b79f006022b8006033b8006fa8970035
:103f7000ffa897000fb197009fb197000dfc0700b5
:103f80000000e0000a003d006fa89700ffa897001e
:103f90000fb197009fb1970003f0a200e0af9f0020
:103fa000f1af9f0082b79f0093b79f003d00b30021
:103fb0000000eb0080a79f006022b8006033b800cb
:103fc0006fa89700ffa897000fb197009fb19700c7
:103fd000fdfb07000000e000340032006fa89700ee
:103fe000ffa897000fb197009fb19700fbfb070058
:103ff00003fc2f000381470023fc07000fa097005c
:104000000000e9006300b900a200200011000900cf
:104010000200d8008000fd0081a79f000100e000a1
:1040200002003d000100e90080a79f000fa4970057
:104030000840ea0029fe07006faa9700ffaa970030
:104040000fb397009fb3970046fb0700a0af9f00f8
:10405000b1af9f00c2af9f00d3af9f006022b800f6
:104060000600200007ff2300d2fb07000000e0004d
:1040700002003d000800e9000b0037006022b80094
:1040800006002000470224002fa89700bfa8970031
:104090004fa99700dfa99700fefb07000000e00092
:1040a000020035000800e80080a79f003fb297009b
:1040b000f80f520057003c00d0c6b300804f5200aa
:1040c000290036000485fb0042062000110009008b
:1040d0000285d80000017800010478004311dd005a
:1040e000ebe520000b0141006022b8000600200033
:1040f00007fe23000288900092889000b289900009
:104100002289900017fb0700a9002000809fbe00b5
:10411000110009000984d800000478004f00be0097
:104120004344dd000b04440048229000d822900054
:1041300068239000f82390000afb0700801f780096
:1041400001027800110009000985d8000102fd0074
:104150004f0078004322dd000b0242005403be00f2
:104160004402be001f0037000480fb00e9e5200088
:10417000ea4f520014003600a2002000110009008e
:104180000280d80000017800010478004311dd00ae
:10419000090141006022b8000600200007fe23004c
:1041a00042209000d2209000f221900062219000e5
:1041b000ecfa07004344dd00090444003802be0065
:1041c0002803be00070037004300dd00090040005f
:1041d0006022b8000600200007fe23005001be0048
:1041e0004000be00dffa07000002be000203be006e
:1041f0006fa89700ffa897000fb197009fb1970095
:10420000a9fb0700e0af9f00f1af9f0082b79f00be
:1042100093b79f000fa49700e90f540015003c00ce
:104220006022b8006033b8006fa89700ffa897001d
:104230000fb197009fb1970063fb07000000e000fb
:10424000320032006fa89700ffa897000fb19700c7
:104250009fb1970011fc0700e00f5000e08f58005d
:10426000e00f5900e08f590028003a00e10f540098
:10427000260034000400200005002e00b6e02200d5
:10428000170124002fa89700bfa897004fa99700f7
:10429000dfa9970047fb07000000e00002003d0097
:1042a00073005400010037007200540080a79f0083
:1042b0000fc0970089fd0700a0af9f00b1af9f001e
:1042c000c2af9f00d3af9f000002be000203be003a
:1042d0006fa89700ffa897000fb197009fb19700b4
:1042e0001ffc0700edfb07000205be000004be0036
:1042f0006000b8006011b800a0a79f00b1a79f00a0
:10430000c2a79f00d3a79f002e0037006fa8970079
:10431000ffa897000fb197009fb19700dffb070040
:104320000205be000004be00e00f5000e08f580000
:10433000e00f5900e08f59000200350062fc0700d1
:104340001300370010002000010020006011b800a9
:1043500008006000898060000a0161008b816100b3
:104360008b03d1000a83d3008982d3000882d30053
:10437000000072008180720002017300838173006b
:1043800051fc07000002be000203be0046fb07000e
:104390000002be000203be006fa89700ffa89700ae
:1043a0000fb197009fb197007efc0700a0a79f0068
:1043b000b1a79f00c2a79f00d3a79f000000eb00fa
:1043c00080a79f0014c0b300e5fb20000b0037005e
:1043d0000400fb004300dd00050040005001be006a
:1043e0004000be000040e10001c8e10002d0e10051
:1043f00003d8e100030039000442e800f44f520002
:10440000f3ff3a00c47f9f000400fb00bfb0970099
:10441000008040008fa09700010040004fb197003e
:1044200000075100bfb197000300e0000100320017
:104430000e07e90063806600010032000e07e90004
:104440000d28a30026003200e18066000d18a300ad
:104450000c003200d00220000100e00001003a0010
:104460000080e900efb0970071020700e10f400003
:10447000180032002fb297000402e800a4b79f0092
:10448000140037000100e00012003200efb0970086
:104490000002200066020700e10f40000d0032001c
:1044a000afb297008502e800a5b79f00090037006a
:1044b000efb09700000320005d020700e10f40000d
:1044c000030032002fb697000c06e800acb79f003f
:1044d0000e07e9000e00e000f5ff3c003d0037004c
:1044e0000d38a3000a0032000b003700efb0970030
:1044f000000220004e020700e10f400003003200de
:104500002fb097000000e800a0b79f000e07e90059
:104510000e00e000f5ff3c00e18066000d18a300ee
:104520000c003200d00220000100e00001003a003f
:104530000080e900efb097003d020700e10f400066
:1045400024003200afb097008100e800a1b79f00bf
:10455000200037000100e0001e003200efb097009d
:104560000002200032020700e10f40001900320073
:104570002fb197000201e800a2b79f001500370095
:104580000000fb004300dd00e1fb200001004000d3
:104590003002be002003be000800be000a01be00bb
:1045a0005ff90700a4002000050020006033b80078
:1045b00062f907000003b000efb097001c0207008b
:1045c000e10f400003003200afb197008301e80023
:1045d000a3b79f004f7a97000440e900c07f9f0077
:1045e000e14f4000e6ff3a000b003700efb09700c4
:1045f000000320000e020700e10f4000030032001c
:10460000afb297008502e800a5b79f000fa0970002
:104610000000e90080a79f000fa097000000e000c5
:10462000f2ff3c003fb6970020c1b300f20f5600e6
:1046300001003c006fe09700c07f9f00cf7897009b
:104640000100fb003fb1970000005100e0a79f0070
:104650000104e00008003200efb09700e002200003
:10466000f3010700e10f400003003200afb19700f3
:104670008301e800a3b79f004f78970097fc0700dd
:104680000002be000203be002fa09700bfa097004b
:104690004fa19700dfa19700b2f90700fffa0700ca
:1046a0001e0037000000fb004300dd00ecfb200093
:1046b0000c0040003002be002003be000800be0017
:1046c0000a01be0016f90700a40020000500200022
:1046d0006033b80019f907000003b000efb097008d
:1046e000d3010700e10f4000030032002fb2970012
:1046f0000402e800a4b79f00cf7a97000500fb00f2
:104700004300dd000c0040003002be002003be006c
:104710000800be000a01be0008f907000205be003d
:104720000004be004f7e97000c40e900c07f9f0050
:10473000e14f4000dbff3a000006eb0009003700c4
:10474000efb0970000032000b9010700e10f40001f
:10475000030032002fb097000000e800a0b79f00d0
:104760000c06e800efa09700810f5600f4ff3a0016
:104770000d38a300a10132000e00e0009f013400bb
:104780000006eb00efb0970000022000a801070030
:10479000e10f4000030032002fb197000201e80052
:1047a000a2b79f000c06e8008e0f5600930132005e
:1047b000f4ff37000d007800000cb20028003a002a
:1047c0000d00e00005003d008fb997004305be00d5
:1047d0004304be0083bf9f00140037000d48a300b0
:1047e0000b0032000fba97004400be0084bf9f0048
:1047f0004f89de00cf91de000002be000203780088
:10480000820378000605be000404be0007003700de
:104810008fba97004500780085bf9f00000478009c
:10482000cfc4de00090578008a057800e00f540047
:10483000e08f5c00e00f5d00e08f5d0020003d0038
:104840003d00b3006000b8006011b80008045000db
:10485000898458000a0559008b85590018003700d3
:104860000d00e00005003d000fbe97004c05be00a6
:104870004c04be008cbf9f00110037000d48a30000
:10488000080032008fba97004500be0085bf9f0028
:1048900004017800840178000205be000004be0017
:1048a000070037000fbe97004c0078008cbf9f00b8
:1048b00000047800090020000a0020000b002000fe
:1048c0003fb097000000e00007003a00e00f5400fe
:1048d000e08f5c00e00f5d00e08f5d0002003a00b9
:1048e00011002000b1b79f000d0778000e0cb20038
:1048f00000042000800f57002f00320003003c000e
:104900000e00e000070032003f00370000082000e2
:10491000800f570014003200000c2000800f570059
:1049200039003a0014c0b300e5fb20000b0037004b
:104930000400fb004300dd00050040005001be0004
:104940004000be000040e10001c8e10002d0e100eb
:1049500003d8e1002b0039000442e800f44f520074
:10496000f3ff3a002700370000012000010020007b
:104970006011b80014c0b3000040e10001c8e100bc
:1049800002d0e10003d8e1001e00390045002000fc
:104990000000d0008180d2000281d2008381d20049
:1049a0008502e900faff3a000442e800f04f5200a5
:1049b000f1ff3a00130037008000200001002000c2
:1049c0006011b80014c0b3000040e10001c8e1006c
:1049d00002d0e10003d8e1000a0039003c002000c9
:1049e0000000d0008180d2000281d2008381d200f9
:1049f0000c06e900faff3a000442e800f54f5200c5
:104a0000f1ff3a00c47f9f00cf7897000100fb00c0
:104a10003fb19700820f500002003d00c27f9f000f
:104a200004003700bfb19700808f510001003d00a6
:104a3000b0b79f004fb297000400e00004003200be
:104a400063806600020032000402e900c4b79f00e0
:104a50000de8a3000b003200cfb297003fb69700dd
:104a60008c8f520003003c000000eb00c0b79f0099
:104a700004003700cfb097003fb19700828050000c
:104a8000c1b79f00cf7997000300fb000002eb0045
:104a900094a79f00cfb29700808f5200020034008d
:104aa0000080520090a79f000d28a300370032001d
:104ab000e18066000d18a3000c003200d002200037
:104ac0000100e00001003a000080e900efb097002b
:104ad000d7000700e10f40000e0032002fb697000c
:104ae0000c06e800acb79f000a0037000100e000a8
:104af00008003200efb0970000022000cc00070051
:104b0000e10f4000030032002fb097000000e800e2
:104b1000a0b79f009fa097000100e0000f003200a7
:104b20000006eb00efb0970000032000c000070074
:104b3000e10f4000030032002fb197000201e800ae
:104b4000a2b79f000c06e8009fa19700830f5600b4
:104b5000f4ff3a000002eb0094a79f00bfb2970059
:104b6000c328dd0060fb20008080400091af9f00e3
:104b70004228dd006400500080af9f006328b90028
:104b8000f0a79f0063065000820037001fa6970021
:104b90000c00e00011003200688066000f003a004f
:104ba00000067800efb0970000022000a000070088
:104bb000e10f4000030032002fb097000000e80032
:104bc000a0b79f000c06e8009fa09700810f560039
:104bd000f4ff3a000001eb0092a79f00e18066001d
:104be0000d18a3000c003200d00220000100e000ec
:104bf00001003a000080e900efb097008c00070048
:104c0000e10f4000d5ff3200afb197008301e8000b
:104c1000a3b79f00d1ff37000100e000cfff3200b3
:104c2000efb097000002200081000700e10f400074
:104c3000caff32002fb297000402e800a4b79f0019
:104c4000c6ff370000042000800f570030003200fc
:104c500003003c000e00e000070032003d0037007a
:104c600000082000800f570011003200000c2000c7
:104c7000800f570037003a001fa897003002be008f
:104c80002003be000800be000a01be00a4f7070012
:104c9000a4002000050020006033b800a7f707003b
:104ca00004c3b30004424000c47f9f0029003700c2
:104cb00055062100d5b79f000d58a30002003a0009
:104cc00060072100d0b79f001400200005002000dd
:104cd0006033b8008fa897008100e9000500330019
:104ce0000402d0008582d2000683d2008783d200de
:104cf000f9ff37000800be000a01be0088f7070070
:104d00006f0060005fb197006240780010003700cc
:104d100014002000050020006033b8008c017800ea
:104d20008301e900050033000402d0008582d2002f
:104d30000683d2008783d200f9ff37000800be0047
:104d40000a01be0076f70700674060000043b0002c
:104d5000c07f9f004f7a97000400fb00efb09700e0
:104d600033000700e10f400003003200afb29700ac
:104d70008502e800a5b79f001fa8970068005000b3
:104d800090af9f008fa89700e480500081af9f00f4
:104d900063065600d0ff2f003fb197000090b90086
:104da000ffa197000080410063005000800f560073
:104db000a4ff3a000d38a300100032001fa2970094
:104dc0000400e0000d0034000006eb00efb0970097
:104dd0000002200016000700e10f4000030032002f
:104de000afb297008502e800a5b79f000c06e80067
:104df0001fa09700800f5600f4ff3a007fb1970084
:104e0000b2407800f2b79f00c17f9f000104e0002c
:104e100014fb3a002fb097004f0778004f06be00f2
:104e20004f05be004f04be008f03b1000000060016
:104e3000889fbe000001780001047800b100900056
:104e40000118a3003d0032000198a30003003a00be
:104e5000180090000000e00038003a000190a00027
:104e60003104980082047800f90fb2001800900015
:104e70000000e00002003a0028009000000c7800da
:104e8000ea8f540006003a00380090000078a30032
:104e900003003a0088007800d0002000e4ff0700fb
:104ea0009800900058009000808f50000b00320056
:104eb0000100e800100498001800780009587800f4
:104ec000000c780011c0b300200b210001487800cd
:104ed000ea8f54000600320019003700880078007d
:104ee000094078001900070080047800140037009a
:104ef000380090000088a3001100320018019000d3
:104f0000a80090004800900086f2070098009000ea
:104f1000810f500004003200380090000003b300fd
:104f2000300498008084eb000000eb00100498002f
:104f300028009000000c7800010037008084eb000e
:104f4000090078004f04be00000006000200fa00cd
:104f5000889fbe00a0ff9f0001047800b100900070
:104f6000810478000904b200020032000000fb0056
:104f7000360037000118a30005003a000103b30012
:104f800031049800190498000080eb002f003700ce
:104f9000580090000000e00006003a004800900031
:104fa00012002000e68057005ef207001904980006
:104fb00024003700280090000000e00008003a00bc
:104fc000e00a210020049800000c78002000200056
:104fd00050049800100498000130a000310498009b
:104fe00018019000a8009000480090004df20700c2
:104ff00028009000000c78000080eb00100498005e
:1050000018007800aff8970001587800000c78007d
:105010002ff89700ea4f50000a003a00380090003d
:105020000088a3000700320018019000a80090003b
:10503000480090003bf2070019049800a800900077
:10504000010c7800aff897000100fb004f04be0090
:085050000080fa0000000600d8
:020000040000fa
:0200000401f009
:04000c00fbff0000f6
:020000040000fa
:0200000401f009
:04001000bcff000031
:020000040000fa
:0200000401f009
:04001800ffff0000e6
:020000040000fa
:100008009e6900009e6900009e6900009e690000cc
:100018009e6900009e6900009e6900009e690000bc
:100028009e6900009e6900009e690000e062000071
:100038009e6900009e6900009e6900009e6900009c
:100048009e6900009e6900009e690000bc5f000078
:10005800545f00009e6900009e6900009e690000d0
:100068009e6900009e6900009e6900009e6900006c
:100078009e6900009e6900009e6900009e6900005c
:100088009e6900009e6900009e6900009e6900004c
:100098005c6300009e6900009e690000885f0000a4
:1000a8009e6900009e6900009e6900009e6900002c
:1000b8009e6900009e6900009e6900009e6900001c
:1000c8009e6900009e6900009e6900009e6900000c
:1000d8009e6900009e6900009e6900009e690000fc
:1000e8009e6900009e6900009e6900009e690000ec
:1000f800ae6400009e6900009e6900009e690000d1
:100108009e6900009e6900009e6900009e690000cb
:100118009e6900009e6900009e6900009e690000bb
:100128009e6900009e6900009e6900009e690000ab
:100138009e6900009e6900009e6900009e6900009b
:100148009e6900009e6900009e6900009e6900008b
:100158009e6900009e6900009e6900009e6900007b
:100168009e6900009e6900009e6900009e6900006b
:100178009e6900009e6900009e6900009e6900005b
:100188009e6900009e6900009e6900009e6900004b
:100198009e6900009e6900009e6900009e6900003b
:1001a8009e6900009e6900009e6900009e6900002b
:1001b8009e6900009e6900009e6900009e6900001b
:1001c8009e6900009e6900009e6900009e6900000b
:1001d8009e6900009e6900009e6900009e690000fb
:1001e8009e6900009e6900009e6900009e690000eb
:0801f8009e6900009e690000f1
:020000040000fa
:100208009e6900009e6900009e6900009e690000ca
:100218009e6900009e6900009e6900009e690000ba
:100228009e6900009e6900009e690000e06200006f
:100238009e6900009e6900009e6900009e6900009a
:100248009e6900009e6900009e690000bc5f000076
:10025800545f00009e6900009e6900009e690000ce
:100268009e6900009e6900009e6900009e6900006a
:100278009e6900009e6900009e6900009e6900005a
:100288009e6900009e6900009e6900009e6900004a
:100298005c6300009e6900009e690000885f0000a2
:1002a8009e6900009e6900009e6900009e6900002a
:1002b8009e6900009e6900009e6900009e6900001a
:1002c8009e6900009e6900009e6900009e6900000a
:1002d8009e6900009e6900009e6900009e690000fa
:1002e8009e6900009e6900009e6900009e690000ea
:1002f800ae6400009e6900009e6900009e690000cf
:100308009e6900009e6900009e6900009e690000c9
:100318009e6900009e6900009e6900009e690000b9
:100328009e6900009e6900009e6900009e690000a9
:100338009e6900009e6900009e6900009e69000099
:100348009e6900009e6900009e6900009e69000089
:100358009e6900009e6900009e6900009e69000079
:100368009e6900009e6900009e6900009e69000069
:100378009e6900009e6900009e6900009e69000059
:100388009e6900009e6900009e6900009e69000049
:100398009e6900009e6900009e6900009e69000039
:1003a8009e6900009e6900009e6900009e69000029
:1003b8009e6900009e6900009e6900009e69000019
:1003c8009e6900009e6900009e6900009e69000009
:1003d8009e6900009e6900009e6900009e690000f9
:1003e8009e6900009e6900009e6900009e690000e9
:0803f8009e6900009e690000ef
:020000040000fa
:10505800436500006e740000657200002046000081
:105068007265000071750000656e000063790000cc
:10507800200a000000250000332e000032660000e0
:10508800204d0000487a00000a000000507500001a
:105098006c730000652000004c6500006e6700001e
:1050a80074680000200a000000250000332e00006c
:1050b8003066000020630000796300006c65000022
:1050c8000a000000537400006172000074200000a0
:1050d8004465000070740000682000000a000000a9
:1050e800253300002e300000662000006d6d0000a2
:1050f8000a000000546f0000746100006c2000007a
:105108004465000070740000682000000a00000078
:1051180046690000782000004461000074610000c6
:10512800204d00006f640000652000000a000000a8
:10513800253300002e30000066200000313d0000bd
:105148005452000055450000200a000000460000a7
:1051580069780000205000006f6900006e7400003c
:10516800732000000a000000253300002e300000e4
:105178006620000064610000746100000a000000fd
:1051880045720000726f0000722000005474000025
:105198006c44000070740000680000005052000069
:1051a80046200000200a000000250000332e0000e1
:1051b80030660000204800007a0a00000050000015
:1051c800726500007373000020530000656c0000d6
:1051d8002042000075740000746f00006e2000000b
:1051e8000a000000556c0000747200006173000032
:1051f8006f7500006e640000204300006e740000ac
:10520800726c0000003e00007374000061720000c0
:10521800742000000a0000003e730000746f000054
:10522800702000000a000000776500006c63000031
:105238006f6d0000652000000a00000025330000a3
:105248002e320000662000002020000020200000f0
:105258002020000020200000200a00000045000057
:10526800727200006f72000020280000312d0000cb
:105278003130000029000000253300002e300000e6
:1052880066200000202000002020000020200000d0
:1052980020200000200a0000004500007272000073
:1052a8006f72000020280000312d000025690000e1
:1052b800290000005374000072740000447000005c
:1052c80074680000200a000000540000746c00009c
:1052d800447000007468000020690000732000001a
:1052e8002569000000720000616e0000676500001b
:1052f80020280000302d000025690000290000004a
:10530800547400006c4400007074000068200000b1
:105318000a0000005374000072740000447000001a
:1053280074680000206900007320000025690000ef
:1053380000450000727200006f72000020540000e7
:105348006c7400004470000074680000003e0000a7
:1053580020500000756c000073650000206c000090
:10536800656e000067740000682000006861000036
:105378007320000062650000656e00002063000075
:10538800686100006e67000065640000207400001a
:105398006f20000025690000200d00000a000000b1
:1053a8003e200000505200004620000068610000c6
:1053b8007320000062650000656e00002063000035
:1053c800686100006e6700006564000020740000da
:1053d8006f20000025690000200d00000a00000071
:1053e8003e20000050520000462000004572000098
:1053f800726f00007220000028310000202d00008c
:10540800203200003030000030290000200d00005c
:105418000a000000507200006d740000536c000018
:1054280063740000200a0000003e000020450000d0
:10543800727200006f72000020560000616c00005c
:1054480075650000200d00000a0000003e200000e5
:105458005472000069670000676500007220000050
:10546800736f000075720000636500002073000010
:1054780065740000207400006f200000657800004b
:1054880074650000726e0000616c0000206200000c
:1054980079200000686100007264000077610000f4
:1054a80072650000200d00000a0000003e20000088
:1054b80025690000206f00006620000054470000a6
:1054c8004325000069200000646100007461000049
:1054d80020630000686100006e670000652000001e
:1054e800746f00003a200000003e000020250000f4
:1054f80069200000003e0000200d00000a000000a6
:105508003e200000436500006e74000065720000d4
:10551800204600007265000071750000656e00008d
:10552800637900002020000045720000726f0000bf
:105538007220000028310000202d000020310000da
:1055480030290000200d00000a0000003e20000065
:1055580054720000616e0000736d000069740000f1
:1055680020500000756c000073650000204c00009e
:10557800656e000067740000682000006861000024
:105588007320000062650000656e00002063000063
:10559800686100006e670000656400002074000008
:1055a8006f20000025690000200d00000a0000009f
:1055b8003e200000507500006c730000652000005c
:1055c8004c6500006e67000074680000206d0000e4
:1055d80075730000742000006265000020660000fa
:1055e800726f00006d20000031200000746f000011
:1055f80020250000692c000020630000686100007d
:105608006e67000065200000505200004620000030
:10561800746f0000206900006e630000726500006e
:105628006173000065200000707500006c73000055
:10563800652000006c6500006e670000746800005b
:10564800200d00000a0000003e20000053740000f6
:10565800617200007420000044650000707400004e
:105668006820000068610000732000006265000087
:10567800656e000020630000686100006e6700002e
:1056880065640000207400006f2000002569000098
:10569800206d00006d2000000d0a0000003e000093
:1056a800205400006f740000616c0000204400006a
:1056b8006570000074680000206900007320000015
:1056c8006c650000737300002074000068610000be
:1056d8006e20000053740000617200007420000006
:1056e8006465000070740000682c000020680000e9
:1056f8006173000020620000656500006e200000f4
:1057080063680000616e00006765000064200000a7
:10571800746f000020250000692000006d6d0000f6
:10572800200d00000a0000003e2000005374000015
:10573800617200007420000044650000707400006d
:1057480068200000726100006e670000653a000082
:1057580020300000207400006f2000002569000040
:10576800206d00006d2000000d0a0000003e0000c2
:10577800205400006f740000616c00002044000099
:105788006570000074680000206800006173000004
:1057980020620000656500006e200000636800005c
:1057a800616e00006765000064200000746f0000ef
:1057b80020250000692000006d6d0000200d00000c
:1057c8000a0000003e2000005374000061720000cf
:1057d8007420000044650000707400006820000018
:1057e80069730000206700007265000061740000a2
:1057f8006572000020740000686100006e200000df
:10580800746f0000746100006c2000006465000083
:1058180070740000682c00002068000061730000ac
:1058280020620000656500006e20000063680000cb
:10583800616e00006765000064200000746f00005e
:1058480020250000692000006d6d0000200d00007b
:105858000a0000003e200000546f00007461000040
:105868006c2000004465000070740000682000008f
:10587800726100006e670000653a00002030000089
:10588800207400006f20000025690000206d0000d2
:105898006d2000000d0a0000003e000020540000aa
:1058a80047430000312000006861000073200000b9
:1058b80062650000656e00002063000068610000fa
:1058c8006e67000065640000207400006f2000000f
:1058d80025690000200d00000a0000003e2000009d
:1058e800544700004331000020760000616c00003e
:1058f8007565000020450000727200006f7200009c
:1059080020280000302000002d2000003235000043
:1059180035290000200d00000a0000003e2000008c
:105928005447000043310000207300006c6f0000f2
:1059380070650000206800006173000020620000ac
:10594800656500006e20000063680000616e00005d
:105958006765000064200000746f000020250000c7
:10596800692000000d0a0000003e000020540000dd
:105978004743000031200000736c00006f70000086
:1059880065200000766100006c750000652000004d
:1059980045720000726f000072200000283000007d
:1059a800202d00002032000035350000292000009d
:1059b8000d0a0000003e000020540000474300008c
:1059c800322000006861000073200000626500005a
:1059d800656e000020630000686100006e670000cb
:1059e80065640000207400006f2000002569000035
:1059f800200d00000a0000003e200000544700006f
:105a08004332000020760000616c000075650000dc
:105a180020450000727200006f720000202800000c
:105a2800302000002d20000032350000352900000c
:105a3800200d00000a0000003e2000005075000004
:105a48006c73000065200000646500006c61000054
:105a58007920000068610000732000006265000082
:105a6800656e000020630000686100006e6700003a
:105a780065640000207400006f20000025690000a4
:105a8800200d00000a0000003e20000045720000c2
:105a9800726f000072200000507500006c730000e7
:105aa80065200000446500006c610000792000005a
:105ab800566100006c750000652000002830000069
:105ac800202d00002032000035350000292000007c
:105ad8000d0a0000003e0000205500006c74000014
:105ae80072610000736f0000756e00006420000092
:105af80053740000617200007465000064200000a7
:105b08000d0a0000003e0000205500006c740000e3
:105b180072610000736f0000756e00006420000061
:105b2800537400006f70000070650000642000006e
:105b38000d0a0000003e0000204300006f6d0000c9
:105b48006d6100006e640000204c00006973000065
:105b5800742000000d0a0000003e00002030000004
:105b68002031000030300000202000004365000094
:105b78006e74000065720000204600007265000027
:105b880071750000656e000063790000200d00004b
:105b98000a0000003e2000003120000031200000f3
:105ba80020500000756c000073650000204c000058
:105bb800656e000067740000682000000d0a000090
:105bc800003e0000203200002032000020200000ab
:105bd80053740000617200007420000044650000e6
:105be8007074000068200000696e0000206d0000dd
:105bf8006d2000000d0a0000003e00002033000068
:105c08002035000030200000546f0000746100004f
:105c18006c200000446500007074000068200000db
:105c2800696e0000206d00006d2000000d0a000064
:105c3800003e00002034000020310000323800000f
:105c48002054000047430000312000004c6500004c
:105c5800766500006c2000000d0a0000003e000080
:105c6800203500002031000030200000544700009b
:105c780043310000205300006c6f00007065000085
:105c8800200d00000a0000003e2000003620000021
:105c98003132000038200000544700004332000031
:105ca800204c000065760000656c0000200d0000a7
:105cb8000a0000003e2000003720000031300000bc
:105cc800205400004743000032200000536c0000bd
:105cd8006f700000652000000d0a0000003e000003
:105ce8002038000020310000303000003020000053
:105cf80050720000662000000d0a0000200000001d
:105d08003e20000061200000537400006172000012
:105d1800742000002020000062200000537400005e
:105d28006f700000200d00000a0000003e200000f7
:105d380063200000312c00002030000020530000b8
:105d480065740000206900006e7400006572000030
:105d58006e6100006c2f000065780000746500001b
:105d6800726e0000616c000020740000726900000f
:105d78006767000065720000200d00000a0000003f
:105d88003e20000064200000302c0000203100007c
:105d98002020000054720000616e0000736600004d
:105da800657200002064000061740000612000003a
:105db800696e00002074000065780000742f0000f0
:105dc800626900006e61000072790000206d0000b9
:105dd8006f640000652000000d0a0000003e00000e
:105de800206500002031000035340000302000001c
:105df800536f0000756e0000642000007665000097
:105e08006c6f00006369000074790000206d000069
:105e18002f7300000d0a0000003e000020660000fd
:105e2800203100002c2000003020000053740000b6
:105e380061720000742f0000537400006f7000003e
:105e48002064000061740000612000007374000089
:105e580072650000616d0000200d00000a0000005e
:105e68003e200000672000003120000032200000a2
:105e780033200000342000003520000036200000c8
:105e880037200000382000003920000031300000a1
:105e980020530000657400002054000047430000b0
:105ea800312000000d0a0000003e000020690000bb
:105eb8002031000020320000203300002034000090
:105ec8002035000020350000203700002053000056
:105ed8006574000020540000474300003220000091
:105ee8000d0a0000003e0000206a0000203100007a
:105ef80030300000204c0000696e0000657300001f
:105f0800207300006b69000070200000666f0000bd
:105f180072200000646100007461000020730000ba
:105f280074720000656100006d0d00000a00000039
:105f38003e2000006b2000005265000073650000e1
:105f480074200000546900006d6500007220000094
:105f58000d0a0000003e0000206c000020520000e6
:105f6800656100006420000050610000726100005b
:105f78006d65000074650000722000000d0a0000c5
:105f8800003e000020410000205200006561000032
:105f98006420000052650000676900007374000007
:105fa80065720000732000000d0a0000003e00002a
:105fb8002042000020540000474300002054000005
:105fc80065730000742000003020000031200000bc
:105fd80032200000332000000d0a0000003e0000bf
:105fe80020430000203000003a5700002031000014
:105ff8003a520000203200003a57000052200000b8
:10600800333a000052730000742000004649000033
:10601800464f0000207400006573000074200000e3
:106028000d0a0000003e000020440000203500005a
:10603800205300006574000020540000474300000e
:106048002047000041500000732000000d0a0000a6
:10605800003e000020450000205600006572000048
:10606800736900006f6e0000204e0000756d00001f
:1060780062650000722000000d0a00002000000088
:106088003e2000004620000035300000302000008f
:106098004461000074610000205000006f69000036
:1060a8006e740000732000000d0a0000200000003c
:1060b8003e20000047200000200d00000a200000bc
:1060c800003e00002054000072690000676700006d
:1060d80065720000207300006f7500007263000095
:1060e8006520000068610000732000006265000000
:1060f800656e0000207300006574000020740000c5
:106108006f2000006578000074650000726e000062
:10611800616c0000206200007920000068610000c6
:10612800726400007761000072650000200d0000b5
:106138000a2000002052000065710000756500000b
:106148007374000020640000656e00006e69000032
:1061580065640000200d00000a0000003e200000d9
:106168005472000069670000676500007220000033
:10617800736f0000757200006365000020680000fe
:106188006173000020620000656500006e20000059
:106198007365000074200000746f0000206900001f
:1061a8006e740000657200006e6100006c200000d3
:1061b8000d0a0000003e0000205400007269000033
:1061c8006767000065720000207300006f750000ab
:1061d8007263000065200000686100007320000001
:1061e80062650000656e00002073000065740000a1
:1061f800207400006f2000006578000074650000be
:10620800726e0000616c0000200d00000a000000a2
:106218003e20000045720000726f000072200000ee
:10622800766100006c750000653a000020310000be
:106238003a200000496e000074650000726e00008c
:10624800616c00003b200000303a0000204500004f
:1062580078740000657200006e6100006c20000018
:106268000d0a0000003e0000205300006574000085
:106278002064000061740000612000007472000056
:10628800616e0000736600006572000020690000fe
:106298006e2000007465000078740000206d000016
:1062a8006f640000652c0000206c0000696e00001f
:1062b80065200000737400006172000074730000b0
:1062c800207700006974000068200000412c00005d
:1062d80020740000657200006d6900006e610000a6
:1062e800746500007320000062790000204c0000f3
:1062f800462000000d0a0000003e00002053000068
:1063080065740000206400006174000061200000d2
:1063180074720000616e0000736600006572000010
:10632800206900006e200000626900006e610000b4
:1063380072790000206d00006f640000652c000079
:10634800206c0000696e0000652000007374000076
:106358006172000074730000207700007469000007
:10636800682000006220000074650000726e000062
:10637800696d000061740000657300002062000010
:1063880079200000302000000d0a0000003e0000c7
:1063980020450000727200006f7200002076000035
:1063a800616c0000756500003a200000303a00007a
:1063b8002074000065780000742c0000206c000038
:1063c800696e0000652000007374000061720000af
:1063d80074730000207700006974000068200000d2
:1063e800412c000020740000657200006d690000f7
:1063f8006e6100007465000073200000627900007f
:10640800204c0000463b0000203100003a200000ec
:10641800626900006e610000727900002c200000a3
:106428006c6900006e650000207300007461000054
:10643800727400007320000077740000696800001f
:106448002062000020740000657200006e69000080
:106458006d6100007465000073200000627900001f
:1064680020300000200d00000a0000003e2000003f
:10647800536f0000756e0000642000007665000010
:106488006c6f0000636900007479000020680000e8
:106498006173000020620000656500006e20000046
:1064a8007365000074200000746f00002025000050
:1064b800692000006d2f0000732000000d0a000005
:1064c800003e000020450000727200006f7200005c
:1064d80020760000616c00007565000020660000f1
:1064e8006f720000205300006f7500006e6400009a
:1064f8002053000070650000656400003a20000029
:10650800302000002d200000313000003030000025
:10651800306d00002f730000200d00000a000000fd
:106528003e200000446100007461000020730000f8
:1065380074720000656100006d2000007374000033
:106548006f70000070650000642000000d0a0000f4
:10655800003e00002044000061740000612000003b
:106568007374000072650000616d00002073000004
:10657800746100007274000065640000200d000062
:106588000a0000003e20000045720000726f000003
:1065980072200000766100006c750000653a00000a
:1065a800203000003a200000537400006f70000093
:1065b8003b200000313a00002053000074610000c5
:1065c80072740000200d00000a0000003e20000048
:1065d8004672000065710000756500006e6300007a
:1065e800793a000020250000332e000032660000b2
:1065f800204d0000487a00003b200000200d0000dc
:106608000a0000003e200000507500006c73000076
:10661800653a000020250000692000000d0a0000ee
:10662800003e00002044000065700000746800000f
:106638003a20000025690000206d00006d20000050
:106648002d20000025690000206d00006d2000004d
:106658000d0a0000003e00002054000047430000df
:10666800312000004c650000766500006c3a00009f
:1066780020250000693b0000205300006c6f0000db
:10668800703a000020250000692000000d0a000073
:10669800003e000020540000474300003220000064
:1066a8004c650000766500006c3a0000202500006b
:1066b800693b0000205300006c6f0000703a000036
:1066c80020250000692000000d0a0000003e00009f
:1066d80020500000524600003a20000025690000c2
:1066e800200d00000a0000003e2000005472000047
:1066f8006967000067650000722000004d6f0000a8
:10670800646500003a20000025690000200d0000a3
:106718000a0000003e20000044610000746100008f
:1067280020540000726100006e730000666500006e
:10673800722000004d6f0000646500003a200000e0
:1067480025690000200d00000a0000003e2000001e
:10675800446100007461000020530000747200005e
:10676800656100006d200000456e00006162000058
:106778006c6500003a20000025690000200d00002b
:106788000a0000003e200000466600005374000026
:106798007346000070670000613d00002569000035
:1067a8003b2000004666000053740000734600005a
:1067b8007067000061500000726500003d25000010
:1067c800693b000020460000665200006443000058
:1067d8006e740000723d0000256900002020000052
:1067e8000d0a0000003e000020460000664c000034
:1067f8006e670000746800003a20000025690000f8
:10680800203b000054470000434e00007073000016
:1068180020250000692000003b20000044630000a0
:106828006d7400004e6d0000627200003a20000096
:106838002569000020200000506e000074730000dd
:10684800527400003a200000253300002e32000068
:10685800662000000d0a0000003e00002030000005
:106868003a570000726b00004d6f0000646500002d
:10687800203100003a460000727100006e430000ab
:106888006e74000072200000323a0000506c000064
:10689800734c00006e67000074200000333a00005b
:1068a800506c0000734400006c7900002034000034
:1068b8003a410000644400006c7900004820000060
:1068c800353a0000466600004c6e00006774000010
:1068d80048200000363a0000466600004c6e000072
:1068e800677400004c200000373a00005472000022
:1068f800677200004d640000203800003a4600002e
:10690800664300006e74000072200000393a0000ef
:1069180020410000644400006c7900004c0d000028
:106928000a0000003e200000413a000046660000d0
:106938005374000073200000423a000046660000cd
:106948005772000048200000433a000046660000e5
:10695800574c0000204400003a46000066520000f0
:1069680048200000453a000046660000524c0000ee
:10697800204600003a460000775600007273000077
:106988006e2000000d0a0000003e000020520000aa
:1069980065670000203000007825000030320000d4
:1069a800783a0000203000007825000030320000de
:1069b800780d00000a0000003e2000005447000047
:1069c800432000007465000073740000206f00000d
:1069d80070740000696f00006e3a00002025000006
:1069e800692000000d0a0000003e0000205700004a
:1069f80072690000746900006e650000204600009e
:106a0800494600004f2000002e2e00002e200000d6
:106a18000d0a0000003e0000205700002030000052
:106a2800782500003032000078200000307800001f
:106a380025300000327800002c200000523a000077
:106a48002030000078250000303200007820000057
:106a58003078000025300000327800002c2000003b
:106a680053740000733a00002030000078250000bd
:106a78003032000078200000290d00000a000000d4
:106a88003e2000005265000061640000696e00004d
:106a98006720000046490000464f0000202e0000f5
:106aa8002e2e0000200d00000a0000003e200000ed
:106ab80046490000464f000020680000617300004e
:106ac80020620000656500006e200000726500000d
:106ad8007365000074210000200d00000a0000000a
:106ae8003e200000433a0000205200006576000076
:106af80031390000204600006562000020350000a2
:106b08002c20000032300000313400002032000018
:106b180030310000332c00002056000048440000ab
:106b28004c20000056650000722000002569000016
:106b3800200d00000a0000003e2000005265000001
:106b480074750000726e000020640000617400001b
:106b5800613a000020250000692000003a2000006a
:106b6800446f0000776e0000536100006d700000f4
:106b78006c6900006e6700003a20000025330000b1
:106b88002e320000662000000d0a0000003e0000c2
:106b9800204900006e760000616c00006964000006
:106ba8002120000044610000746100002072000090
:106bb800616e0000676500003a2000003130000077
:106bc800302000002d31000030300000302000005f
:106bd8000d0a0000003e0000204e00006f2000005b
:106be8005375000063680000204300004d44000016
:106bf800200d00000a00000050200000253300008e
:106c08002e320000662000002569000020250000c3
:106c18006920000025690000202500006920000087
:106c28002569000020250000692000002569000072
:106c380020250000692000002569000020250000ab
:106c4800692000000d0a00000054000047430000be
:106c580020250000692000002569000000200000b0
:106c680025690000002000000d0a00000041000016
:106c78000020000025690000202500006920000090
:106c88000d0a0000003e000020430000656e000071
:106c980074650000722000004672000065710000f3
:106ca800756500006e6300007920000069730000bc
:106cb8002073000065740000207400006f2000003d
:106cc800253300002e320000662000000d0a000067
:106cd800003e0000205400006f740000616c00004a
:106ce80020440000657000007468000020690000fe
:106cf800732000007365000074200000746f0000aa
:106d080020250000692000006d6d00000d0a0000bc
:106d1800003e0000205300007461000072740000ff
:106d280020440000657000007468000020690000bd
:106d3800732000007365000074200000746f000069
:106d480020250000692000006d6d0000200d000066
:106d58000a00000046500000474100002052000091
:106d68006567000069730000746500007220000008
:106d78005465000073740000696e0000672e0000ff
:106d88002e2e0000200d00000a00000052650000b1
:106d98006769000073740000657200002531000007
:106da8006420000045720000726f0000722100002c
:106db8000d0a0000005200006567000069730000ba
:106dc8007465000072250000316400002050000046
:106dd8006173000073650000642e00002e0d000032
:106de8000a000000536f00006e6f00004c61000045
:106df8006220000045630000686f00002049000021
:106e0800200d00000a000000426900006f530000d6
:106e18006f6e00006f200000496e0000632e0000b6
:106e2800202000000d0a0000004900006e690000e3
:106e380074690000616c0000697a0000696e0000e6
:106e48006720000046500000474100000d0a00007e
:106e5800005300007563000063650000656400006e
:106e680065640000200d00000a0000005365000062
:106e7800742000004672000065710000756500000e
:106e88006e63000079200000746f0000203100005c
:106e98004d4800007a2000000d0a0000004600005e
:106ea800616900006c650000642000002a2a000067
:106eb8002a2a00002a2000000d0a00000000000015
:020000040000fa
:106ec8004e00fa00881f780006cebf000000fb00c5
:106ed800602798006e209000e30f50005f0032009a
:106ee800ee209000e38f50000a003c006e209000d6
:106ef800e10f500024003200ee209000e18f500096
:106f080035003c006e2090000000e0000b003200cd
:106f1800c8003700ee209000e58f50009300320043
:106f28006e209000e50f50006d003500ee209000b7
:106f3800e68f5000ab003200be0037001000200082
:106f48001c180700c0822a0032180700506e800003
:106f5800616e8000906d8800a16d8800906d800042
:106f6800a16d8000809fbe00f0832a00801f7800fa
:106f78000e00780040f20700e68757000e00780000
:106f88003c180700af003700100020000918070060
:106f9800a0842a001f180700706e8000cf80de00d2
:106fa80095ea0700906d8800a16d8800906d8000bb
:106fb800a16d8000809fbe0090852a00801f780008
:106fc8000e0078002cf20700e68757000e007800c4
:106fd800281807009b00370010002000f51707004d
:106fe80060862a000b180700586b80006140b900c2
:106ff80081ea070040279800512798000800e00020
:1070080007003d0002002000037824004e20900075
:10701800de209000a4ea0700402798005127980036
:107028004e209000de209000906d8800a16d8800b1
:10703800906d8000a16d8000809fbe0040872a006f
:10704800801f78000e0078000bf20700e6875700d3
:107058000e007800071807007a003700100020009b
:10706800d4170700e0872a00ea170700686b80003a
:107078006140b90060ea070020279800312798008e
:107088000800e00007003d0002002000037824000b
:107098002e209000be20900083ea07002027980049
:1070a800312798002e209000be209000906d880017
:1070b800a16d8800906d8000a16d8000809fbe004a
:1070c80040872a00801f78000e007800eaf1070048
:1070d800e68757000e007800e617070059003700ca
:1070e80010002000b3170700c0882a00c91707003e
:1070f80008de2000184478000800fb00cf80de007e
:107108003dea070000279800112798000804e000ce
:1071180007003d0002002000033824000e209000e4
:107128009e20900060ea0700002798001127980029
:107138000e2090009e209000906d8800a16d880020
:10714800906d8000a16d8000809fbe00c0892a00dc
:10715800801f78000e007800c7f10700e687570007
:107168000e007800c3170700360037001000200013
:1071780090170700b08a2a00a6170700a06b8000a6
:10718800cf80de001cea0700906d8800a16d8800a2
:10719800906d8000a16d80006011b8009fea070023
:1071a8000000e00001003c000b003700906d8000fb
:1071b800a16d8000809fbe00808b2a00801f780010
:1071c8000e007800acf10700e68757000e00780043
:1071d800a81707001b003700408c2a00a5170700d6
:1071e800180037001000200072170700208d2a00b1
:1071f80088170700206e8000cf80de00fee90700b8
:10720800906d8800a16d8800906d8000a16d800050
:10721800809fbe00908d2a00801f78000e007800a5
:1072280095f10700e68757000e00780091170700d0
:1072380004003700100020005e170700308e2a0077
:10724800741707004f0478000080fa000000060059
:107258000200fa002117800000002800008070005a
:107268002017880030178000000f78001e00780073
:107278000000e000160035000040eb00bfedb7004d
:10728800bfcdbf000004e00013003a00becdbf0030
:10729800e14f500010003a0006cebf000004e000a5
:1072a8000700350006cebf00e54f500004003c0043
:1072b80006cebf000040e80006eeb7000200370027
:1072c8000040eb0006eeb700fdfe070002003700a5
:1072d80010c0b300bfedb700bfcdbf00beedb70013
:1072e8000080fa00000006000200fa00b6cdbf00d8
:1072f8000000fb00000f7800100620009e007800b8
:10730800808f500005003200200620009e00780083
:10731800808f50001a00320025003700100020002e
:1073280024170700608f2a003a17070070902a0078
:1073380050170700110020008000200033110700bb
:107348000000000000000000000000000000000035
:107358000000000000000000000000000000000025
:107368000040eb00efedb700210020008000200076
:107378002611070010002000e0688800120037007e
:10738800100020000b170700608f2a002117070044
:1073980000912a00371707000000eb00e06888001a
:1073a8008000eb008000200018110700060037005d
:1073b80010002000ff160700608f2a00151707002d
:1073c80080912a002b1707000080fa0000000600b1
:1073d8000200fa00211780000000240000807000dd
:1073e8002017880030178000000f78001e007800f2
:1073f8004e00de000000a200610060000004e00012
:10740800160032000040eb00bdedb700bdcdbf0057
:107418000004e00013003a00bccdbf00e14f50006b
:1074280010003a0061db20009140780010c6b300dc
:1074380080cf500003003a0020c6b300b6edb70075
:107448000400370020c6b300b6edb70010c6b3007d
:10745800b6edb700a4ff07000200370010c0b30064
:10746800bdedb700bdcdbf00bcedb7000080fa0090
:10747800000006006600fa00881f780021178000c7
:10748800000022000080700020178800301780005c
:10749800000f78001e0078004d00de000000a200fa
:1074a800610060000004e000da0232000040eb00f6
:1074b800c1edb700c1cdbf000004e000d7023a001b
:1074c800c0cdbf00e14f5000d4023a0006cebf0045
:1074d8000000fb00203798002e319000e30f510088
:1074e800550132002e329000e30f52000a003c0092
:1074f8002e309000e10f50004c0032002e319000e9
:10750800e10f51009a003c002e3290000400e00088
:107518000b003200ba0237002e309000e50f500001
:10752800110232002e319000e50f5100ee013500b6
:107538002e329000e60f520054023200b00237009b
:10754800906d8000a16d80000041eb0032e798004b
:1075580032332300f3112400b2e907000000e000f1
:10756800010034000200370014c0b30034e798006b
:107578003ee090000004a2000004e00027003a006a
:10758800906d8000a16d80000041eb0022e798001b
:107598000200200003f82300a0e907000000e00033
:1075a80001003d000200370014c0b30024e7980032
:1075b8002ee090000004a2000004e00017003a004a
:1075c800906d8000a16d8000d2cc2c00c3d4230024
:1075d80035e90700906d8800a16d8800906d8000e6
:1075e800a16d8000506e8800616e8800906d8000eb
:1075f800a16d80000e81e800809fbe0020922a00c5
:10760800801f7800020078009bf00700e68757008b
:107618000e80e800971607000200370030932a0012
:10762800941607002c0f07007c023700226e80009a
:10763800007d2000110009000200d800806e88003b
:10764800806e8000f00f500002003400000120001e
:10765800806e8800806e8000cf80de00e6e807003c
:10766800926d8000a36d80000042eb0014e7980043
:107678006ae907000000e00001003c000200370052
:1076880010c0b30010e798001ee090000004a200ac
:107698000004e00027003a00906d8000a16d800092
:1076a8000041eb0002e798000200200003f82300e5
:1076b8005ae907000000e00001003d000200370021
:1076c80014c0b30004e798000ee090000004a20084
:1076d8000004e00017003a00906d8000a16d800062
:1076e8000200200003f82300efe80700906d8800ef
:1076f800a16d8800906d8000a16d80004be90700a6
:10770800706e8800906d8000a16d80000e81e80089
:10771800809fbe0000942a00801f78000200780035
:1077280055f00700e68757000e80e800511607005d
:107738000a003700806e80008e80e800801f780085
:1077480010952a00801f7800010078004af0070091
:10775800e48757000e80e80046160700706e800028
:107768008000780020002000281007002b02370036
:10777800706b80006a0450006140b9009ee8070001
:10778800602f9800712f98000800e00007003d0066
:1077980002002000037824006e289000fe28900044
:1077a800c1e80700602f9800712f9800926d800043
:1077b800a36d80000040eb0030df98006e28900039
:1077c800fe28900015e907000000e00001003c00d9
:1077d8000200370012c0b30032df98003ed8900094
:1077e8000004a2000004e00084003a00906d8000cc
:1077f800a16d80000042eb0024df98006011b80002
:1078080006e907000000e00001003d000200370023
:1078180010c0b30020df98002ed890000004a2000a
:107828000004e00075003a00906d8000a16d8000b2
:1078380002002000031224009be80700906d8800d6
:10784800a16d8800906d8000a16d800018e9070087
:10785800506b8800906d8000a16d80000e81e8005b
:10786800809fbe0000942a00801f780002007800e4
:1078780001f00700e68757000e80e800fd150700b5
:10788800516b8000606b8000808f500017003600bd
:10789800506b800000004000606b8800616b8000c6
:1078a800706b8000808f500002003600706b800083
:1078b800606b880010002000be150700e0952a00c4
:1078c800d4150700606b80008e80e800801f780068
:1078d80090962a00801f780001007800e6ef0700e4
:1078e800e48757000e80e800e2150700506b80001f
:1078f80000004000000478006140b9003ee807003d
:10790800302f9800412f98000800e00007003d0044
:1079180002002000037824003e289000ce28900022
:1079280061e80700302f9800412f9800926e800080
:10793800a36e80003e289000ce289000f7e807004c
:1079480002002000832c240036e90700d8e807004d
:10795800806b8800616b8000506b80000080500055
:1079680000004000000478006140b90022e80700e8
:10797800102f9800212f98000800e00007003d0014
:1079880002002000037824001e289000ae289000f2
:1079980045e80700102f9800212f9800926e80006c
:1079a800a36e80001e289000ae289000dbe8070038
:1079b80002002000832c24001ae90700bce8070015
:1079c800906b88000040eb00e0edb700906b800002
:1079d800a06b8800d0cc2c00c1dc2300e06e8800ae
:1079e800f16e8800806b8000d0100700906b8000db
:1079f800f8100700df040700880137001000200096
:107a08006c150700e0952a0082150700706b80004e
:107a18008e80e800801f780070972a00801f780009
:107a28000100780094ef0700e48757000e80e80013
:107a38009015070079013700706b80006a045000c8
:107a48006140b900ece7070070279800012f980003
:107a58000800e00007003d00020020000378240031
:107a68007e2090008e2890000fe80700702798006d
:107a7800012f9800926d8000a36d80000042eb00fa
:107a880054cf98007e2090008e28900063e807006d
:107a98000000e00001003c000200370010c0b30005
:107aa80050cf98005ec890000004a2000004e000d7
:107ab8007e003a00906d8000a16d80000041eb00cf
:107ac80042cf98006011b80054e807000000e000b9
:107ad80001003d000200370014c0b30044cf9800f5
:107ae8004ec890000004a2000004e0006f003a00b5
:107af800906d8000a16d8000020020000312240018
:107b0800e9e70700906d8800a16d8800906d8000fe
:107b1800a16d800066e80700606b8800906d8000aa
:107b2800a16d80000e81e800809fbe0000942a00ad
:107b3800801f7800020078004fef0700e6875700a3
:107b48000e80e8004b150700516b8000606b8000c9
:107b5800808f500011003600606b80000000d1005b
:107b6800506b8800100020001215070040982a006a
:107b780028150700506b80008e80e800801f780071
:107b8800e0982a00801f7800010078003aef07008b
:107b9800e48757000e80e80036150700506b800018
:107ba80000004000000478006140b90092e7070037
:107bb80040279800512798000800e00007003d0082
:107bc80002002000037824004e209000de20900060
:107bd800b5e707004027980051279800926e80006b
:107be800a36e80004e209000de2090004be8070036
:107bf80002002000832c24008ae807002ce80700f4
:107c0800806b8800616b8000506b800000805000a2
:107c180000004000000478006140b90076e70700e2
:107c280020279800312798000800e00007003d0051
:107c380002002000037824002e209000be2090002f
:107c480099e707002027980031279800926e800056
:107c5800a36e80002e209000be2090002fe8070021
:107c680002002000832c24006ee8070010e80700bb
:107c7800906b88000040eb00e0edb700906b80004f
:107c8800a06b8800d0cc2c00c1dc2300e06e8800fb
:107c9800f16e8800806b800024100700906b8000d4
:107ca8004c10070033040700dc00370010002000e8
:107cb800c014070040982a00d6140700706b800093
:107cc8008e80e800801f780070972a00801f780057
:107cd80001007800e8ee0700e48757000e80e8000e
:107ce800e4140700cd003700906d8000a16d80007e
:107cf8006011b800cbe707000000e0000100320087
:107d0800c6003700906d8000a16d80000200200041
:107d180003f8230064e70700906d8800a16d8800d0
:107d2800906d8000a16d8000e1e70700e0edb700ed
:107d3800401f2000a06b8800906d8000a16d80001e
:107d48000e81e800809fbe0000942a00801f780002
:107d580002007800c8ee0700e68757000e80e800aa
:107d6800c4140700ad003700e0cdbf000004e000f8
:107d78003a003a00906d8000a16d8000020020005a
:107d880003f8230048e70700906d8800a16d88007c
:107d9800906d8000a16d8000a4e70700a06b8800ab
:107da800a06b800080007800906b8000808f50006e
:107db8000f003e00a06b80000000e0000c003400c3
:107dc800906d8000a16d80000e81e800809fbe004c
:107dd80000942a00801f780002007800a6ee0700b1
:107de800e68757000e80e800a21407008b003700d2
:107df800a06b800080007800906b8000808f50001e
:107e080013003600906b8000a06b8800a06b800088
:107e1800cf80de00f8e60700906d8800a16d88002d
:107e2800906d8000a16d80000e81e800809fbe00eb
:107e380000942a00801f7800020078008eee070068
:107e4800e68757000e80e8008a14070073003700a1
:107e5800d0992a008714070070003700906d8000c1
:107e6800a16d80000e81e800809fbe0000942a006a
:107e7800801f7800020078007fee0700e687570031
:107e88000e80e8007b14070064003700906d8000c6
:107e9800a16d80000041eb0032c79800020020006d
:107ea800a34f24005fe707000000e0000100340052
:107eb8000200370014c0b30034c798003ec09000d9
:107ec8000004a2000004e0004a003a00906d80001f
:107ed800a16d80000041eb0022c79800020020003d
:107ee80003f823004de707000000e00001003d0013
:107ef8000200370014c0b30024c798002ec09000b9
:107f08000004a2000004e0003a003a00906d8000ee
:107f1800a16d800045e70700206e8800226e800072
:107f2800007d2000110009000200d800806e880042
:107f3800806e8000f00f5000020034000001200025
:107f4800806e8800816e8000706e8000808f500087
:107f580010003d00806e8000706e8800706e80009a
:107f68008000780020002000280e0700706e800036
:107f78008e80e800801f7800b09a2a00801f780061
:107f8800010078003cee0700e48757000e80e80007
:107f98003f110700206e800045120700206e800008
:107fa8008e80e800801f7800409d2a00801f78009e
:107fb8000100780030ee0700e48757000e80e800e3
:107fc80033110700906d8000a16d80000e81e800dc
:107fd800809fbe0000942a00801f7800020078006d
:107fe80025ee0700e68757000e80e80021140700f9
:107ff8000a003700409f2a002511070007003700b4
:1080080010002000eb130700e0a02a00011407006d
:108018000200370010c0b300c1edb700c1cdbf00ea
:10802800c0edb7004f0478000080fa000000060099
:108038006600fa00881f78002117800000002100e0
:10804800008070002017880030178000000f78002b
:108058001e0078004c00de000000a20061006000f5
:108068000004e000db0232000040eb00c3edb70083
:10807800c3cdbf000004e000d8023a00c2cdbf0063
:10808800e14f5000d5023a0006cebf000000fb00c9
:10809800203798002e319000e30f5100550132002f
:1080a8002e329000e30f52000a003c002e30900060
:1080b800e10f50004c0032002e319000e10f5100ca
:1080c8009a003c002e3290000400e0000b003200c1
:1080d800bb0237002e309000e50f5000120232002c
:1080e8002e319000e50f5100ee0135002e32900040
:1080f800e60f520055023200b1023700906d800041
:10810800a16d80000041eb0032e7980002002000da
:1081180003122400c3e607000000e0000100340059
:108128000200370014c0b30034e798003ee0900026
:108138000004a2000004e00027003a00906d8000cf
:10814800a16d80000041eb0022e7980062662600de
:1081580063f82300b1e607000000e00001003d00dd
:108168000200370014c0b30024e798002ee0900006
:108178000004a2000004e00017003a00906d80009f
:10818800a16d8000d2cc2c00c3d4230045e60700a3
:10819800906d8800a16d8800906d8000a16d8000b1
:1081a800506e8800616e8800906d8000a16d80001f
:1081b8000e81e800809fbe0020922a00801f780070
:1081c80002007800aced0700e68757000e80e80053
:1081d800a81307000200370030932a00a5130700f0
:1081e8003d0c07007d023700226e8000007d2000d4
:1081f800110009000200d800806e8800806e80009f
:10820800f00f50000200340000012000806e88004a
:10821800806e8000cf80de00f7e50700926d800059
:10822800a36d80000042eb0014e798007be607008e
:108238000000e00001003d000200370010c0b3005c
:1082480010e798001ee090000004a2000004e0007f
:1082580027003a00906d8000a16d80000041eb007e
:1082680002e798000200200003f823006be60700ed
:108278000000e00001003c000200370014c0b30019
:1082880004e798000ee090000004a2000004e0005b
:1082980017003a00906d8000a16d80000200200058
:1082a80003f82300ffe50700906d8800a16d8800a2
:1082b800906d8000a16d80005ce60700706e8800fc
:1082c800906d8000a16d80000e81e800809fbe0047
:1082d80000942a00801f78000200780066ed0700ed
:1082e800e68757000e80e800621307000a0037008f
:1082f800806e80008e80e800801f780010952a002c
:10830800801f7800010078005bed0700e4875700c4
:108318000e80e80057130700706e80008000780018
:1083280020002000390d07002c023700786b8000f0
:108338006140b900b0e50700602f9800712f9800e0
:108348000800e00007003d00020020000378240038
:108358006e289000fe289000d3e50700602f980053
:10836800712f9800926d8000a36d80000040eb0093
:1083780030df98006e289000fe28900027e607005e
:108388000000e00001003d000200370012c0b30009
:1083980032df98003ed890000004a2000004e000fc
:1083a80085003a00906d8000a16d80000042eb00ce
:1083b80024df9800020020000313240017e60700ba
:1083c8000000e00001003c000200370010c0b300cc
:1083d80020df98002ed890000004a2000004e000de
:1083e80075003a00906d8000a16d800002002000a9
:1083f80003122400abe50700906d8800a16d88008a
:10840800906d8000a16d800029e60700506b880000
:10841800906d8000a16d80000e81e800809fbe00f5
:1084280000942a00801f78000200780012ed0700ef
:10843800e68757000e80e8000e130700516b800096
:10844800606b8000808f500017003600506b8000f2
:1084580000004000606b8800616b8000706b8000da
:10846800808f500002003600706b8000606b8800bf
:1084780010002000cf120700e0952a00e51207003f
:10848800606b80008e80e800801f780090962a003c
:10849800801f780001007800f7ec0700e487570098
:1084a8000e80e800f3120700506b800000004000c7
:1084b800000478006140b9004fe50700302f9800ac
:1084c800412f98000800e00007003d00020020004e
:1084d800037824003e289000ce28900072e507001b
:1084e800302f9800412f9800926e8000a36e800074
:1084f8003e289000ce28900008e6070002002000e1
:10850800832c240047e60700e9e50700806b880014
:10851800616b8000506b80000080500000004000bc
:10852800000478006140b90033e50700102f980077
:10853800212f98000800e00007003d0002002000fd
:10854800037824001e289000ae28900056e5070006
:10855800102f9800212f9800926e8000a36e800043
:108568001e289000ae289000ece5070002002000cd
:10857800832c24002be60700cde50700906b8800cc
:108588000040eb00e0edb700906b8000a06b880026
:10859800d0cc2c00c1dc2300e06e8800f16e88008e
:1085a800806b8000e10d0700906b8000090e0700ca
:1085b800f001070089013700100020007d12070034
:1085c800e0952a0093120700706b80008e80e80007
:1085d800801f780070972a00801f780001007800bb
:1085e800a5ec0700e48757000e80e800a1120700f9
:1085f8007a013700786b80006140b900fee407001b
:1086080070279800012f98000800e00007003d003f
:1086180002002000037824007e2090008e2890001d
:1086280021e5070070279800012f9800926d8000bf
:10863800a36d80000042eb0054cf98007e2090008c
:108648008e28900075e507000000e00001003d005d
:108658000200370010c0b30050cf98005ec89000e9
:108668000004a2000004e0007f003a00906d800042
:10867800a16d80000041eb0042cf9800020020006d
:108688000313240065e507000000e00001003c003a
:108698000200370014c0b30044cf98004ec89000c1
:1086a8000004a2000004e0006f003a00906d800012
:1086b800a16d80000200200003122400f9e40700e5
:1086c800906d8800a16d8800906d8000a16d80007c
:1086d80077e50700606b8800906d8000a16d8000d1
:1086e8000e81e800809fbe0000942a00801f780059
:1086f8000200780060ec0700e68757000e80e8006b
:108708005c120700516b8000606b8000808f500006
:1087180011003600606b80000000d100506b8800ab
:10872800100020002312070040982a003912070081
:10873800506b80008e80e800801f7800e0982a0047
:10874800801f7800010078004bec0700e487570091
:108758000e80e80047120700506b800000004000c0
:10876800000478006140b900a3e40700402798009e
:10877800512798000800e00007003d000200200093
:10878800037824004e209000de209000c6e4070005
:108798004027980051279800926e8000a36e8000b1
:1087a8004e209000de2090005ce5070002002000cb
:1087b800832c24009be507003de50700806b8800bb
:1087c800616b8000506b800000805000000040000a
:1087d800000478006140b90087e40700202798006a
:1087e800312798000800e00007003d000200200043
:1087f800037824002e209000be209000aae40700f1
:108808002027980031279800926e8000a36e800080
:108818002e209000be20900040e5070002002000b6
:10882800832c24007fe5070021e50700906b880072
:108838000040eb00e0edb700906b8000a06b880073
:10884800d0cc2c00c1dc2300e06e8800f16e8800db
:10885800806b8000350d0700906b80005d0d070070
:1088680044010700dd00370010002000d111070087
:1088780040982a00e7110700706b80008e80e8009e
:10888800801f780070972a00801f78000100780008
:10889800f9eb0700e48757000e80e800f5110700a0
:1088a800ce003700906d8000a16d8000020020008e
:1088b80003f82300dbe407000000e00001003200b9
:1088c800c6003700906d8000a16d80000200200076
:1088d80003f8230073e40700906d8800a16d8800f9
:1088e800906d8000a16d8000f1e40700e0edb70015
:1088f800906b8000a06b8800906d8000a16d800057
:108908000e81e800809fbe0000942a00801f780036
:1089180002007800d8eb0700e68757000e80e800d1
:10892800d4110700ad003700e0cdbf000004e0001f
:108938003a003a00906d8000a16d8000020020008e
:1089480003f8230057e40700906d8800a16d8800a4
:10895800906d8000a16d8000b4e40700a06b8800d2
:10896800a06b800080007800906b8000808f5000a2
:108978000f003e00a06b8000e10f50000c00340097
:10898800906d8000a16d80000e81e800809fbe0080
:1089980000942a00801f780002007800b6eb0700d8
:1089a800e68757000e80e800b21107008b003700f9
:1089b800a06b800080007800906b8000808f500052
:1089c80013003600906b8000a06b8800a06b8000bd
:1089d800cf80de0008e40700906d8800a16d880054
:1089e800906d8000a16d80000e81e800809fbe0020
:1089f80000942a00801f7800020078009eeb070090
:108a0800e68757000e80e8009a11070073003700c8
:108a1800d0992a009711070070003700906d8000e8
:108a2800a16d80000e81e800809fbe0000942a009e
:108a3800801f7800020078008feb0700e687570058
:108a48000e80e8008b11070064003700906d8000ed
:108a5800a16d80000041eb0032c7980002002000a1
:108a6800a34f24006fe407000000e0000100340079
:108a78000200370014c0b30034c798003ec090000d
:108a88000004a2000004e0004a003a00906d800053
:108a9800a16d80000041eb0022c798000200200071
:108aa80003f823005de407000000e00001003d003a
:108ab8000200370014c0b30024c798002ec09000ed
:108ac8000004a2000004e0003a003a00906d800023
:108ad800a16d800055e40700206e8800226e80009a
:108ae800007d2000110009000200d800806e880077
:108af800806e8000f00f500002003400000120005a
:108b0800806e8800816e8000706e8000808f5000bb
:108b180010003d00806e8000706e8800706e8000ce
:108b28008000780020002000380b0700706e80005d
:108b38008e80e800801f7800b09a2a00801f780095
:108b4800010078004ceb0700e48757000e80e8002e
:108b58004f0e0700206e8000550f0700206e800022
:108b68008e80e800801f7800409d2a00801f7800d2
:108b78000100780040eb0700e48757000e80e8000a
:108b8800430e0700906d8000a16d80000e81e80003
:108b9800809fbe0000942a00801f780002007800a1
:108ba80035eb0700e68757000e80e8003111070013
:108bb8000a003700409f2a00350e070007003700db
:108bc80010002000fb100700e0a02a001111070088
:108bd8000200370010c0b300c3edb700c3cdbf001b
:108be800c2edb7004f0478000080fa0000000600cc
:108bf8000600fa000000eb00100798002000200093
:108c0800000f7800290037009e00780010e120004e
:108c18000080400090407800f0c2b30080cf500040
:108c2800160036009e00780010e120000080400009
:108c38009040780090c3b30080cf50000f003e00f2
:108c48001e0090006a00b900100798009e00780086
:108c580010e1200000804000104078008080fb0078
:108c68001e0090008080400000fd2f000080400022
:108c7800100798001e0fe8000c0037009e007800cf
:108c880010e12000008040009040780000c2b3004e
:108c980080cf50000200320090a12a00fc0d07008e
:108ca8000080eb00200798000e0037009e00780037
:108cb80010e120000080400010407800ed4f500087
:108cc800060032009e00780010e12000008040007d
:108cd80010407800ea4f5000cbff3a001e00900089
:108ce800200798002e0090000080fa00000006007f
:108cf8000200fa002a83a800011680000000210063
:108d0800008070000016880010168000000f7800a0
:108d18001e0078004c00de00610060000004e000e6
:108d28000300320010002000906f88000f00370009
:108d38000000eb00906f8800c5a2a800c1a2a9009e
:108d4800a06f8000e10f500004003a000000eb0023
:108d5800a06f8800a0a22a00cd0d0700a06f800098
:108d68008000780070002000a80a07000080fa0040
:108d7800000006001400fa00889fbe00606b8000a7
:108d880000004000000478006140b9001ae30700c1
:108d9800000f9800110f98000800e00007003d0040
:108da80002002000037824000e0890009e0890001e
:108db8003de30700000f9800110f9800926e8000a5
:108dc800a36e80000e0890009e089000d3e3070071
:108dd8000004be00f9cdbf000080fb00cf80de009c
:108de80005e307006266260063002c000de4070017
:108df8000001be000800be002be307000004be000f
:108e0800f9cdbf000080fb00cf80de00fae207004a
:108e1800a299290093e1230002e407000001be00a3
:108e28000800be00bde3070080e30700007088006b
:108e38000000eb00000f780070003700facdbf008b
:108e48008081fb00f9cdbf000080fb000000d1004d
:108e58000080fb009e001000fccdbf000080fb00de
:108e68000088b90080007800f9cdbf000081fb00c0
:108e7800110009008200d800000040000080410075
:108e8800100798001e0090000000e00002003d005e
:108e98000000eb00100798009e009000f00f2000e3
:108ea800808f500002003400f00f20001007980057
:108eb8001e0178001e0090008040780090d82000a5
:108ec8000000410001487800fbcdbf000080fb0096
:108ed800cf80de00c8e2070060079800710798009d
:108ee8001e007800cf80de00c3e207000004be0049
:108ef800f9cdbf000080fb00cf80de00bee2070096
:108f08000200200003002c0084e307000001be00db
:108f18000800be00e4e207004007980051079800e7
:108f2800d8df2000184478000800fb00cf80de005e
:108f3800b1e2070020079800310798000804e00014
:108f480007003d0002002000033824002e00900096
:108f5800be009000d4e2070020079800310798006f
:108f68002e019000be0190004e009000de0090009f
:108f7800ace307000004be00f9cdbf000080fb0091
:108f8800cf80de009ce207000001be000800be00a2
:108f980062e307000001be00c3e207000001be0053
:108fa8006e009000fe009000bfe207001fe307007c
:108fb800100798001e0090000000e00002003d002d
:108fc8000000eb00100798009e009000f00f2000b2
:108fd800808f500002003400f00f20001007980026
:108fe8001e0178001e00900080407800d0d9200033
:108ff80000004100014878001e0fe800f9cdbf00cd
:109008000080fb009e0f50008cff3c004f04be0008
:109018000080fa00000006000800fa002007980007
:10902800310798006000b800008fbe0008003700c4
:109038000000000000000000000000000000000028
:1090480010002000010020001e0f40005e9748001d
:109058002e009000be009000be0f1000ae8f1800ca
:10906800f3ff39000080fa00000006007200fa00e1
:10907800003f98000000eb00300798002000200017
:10908800100798000000eb00000f78008104200012
:109098008e8040000000eb00800878005200370006
:1090a8009e00900010e12000008040009040780071
:1090b800f0c2b30080cf5000260036009e0090001a
:1090c80010e12000008040009040780090c3b30079
:1090d80080cf50001f003e00be0190003e0090006f
:1090e800810420008e8040000000400060807800ed
:1090f8006a00b90000017800810420008e804000d9
:109108000380410002b07800be0190003e0090004c
:10911800810420008e8040000000400060817800bb
:109128009e00900010e12000008040001040780070
:109138000080fb008000410000fd2f0000814000fe
:10914800810420008e8040000380410002b0780036
:10915800220037009e00900010e1200000804000af
:109168009040780000c2b30080cf50000a003a0057
:109178003e0090000000e800300798003e00900094
:10918800820420000e014100800040000000eb0036
:1091980080307900110037009e00900010e1200017
:1091a8000080400010407800ea4f500007003a0065
:1091b8009e00900010e12000008040009040780060
:1091c80000c2b30080cf50000400320090a12a00f2
:1091d800af0c070010002000000f78001e00900060
:1091e8000000e800100798009e00900010e12000a1
:1091f8000080400010407800ed4f5000a8ff3a0072
:109208001e00e0003e003a00e80047000e389000db
:10921800801f78003e009000801f7800a0a52a00db
:10922800801f78000100780093e90700e68757005f
:1092380068004700960c07000000eb002007980024
:10924800290037000e389000e10f50000b003a005b
:109258002e0190002e009000810420008e80400096
:1092680000004000608078008040780090d820009e
:1092780000004100014878000a0037002e019000e4
:109288002e009000810420008e80400000004000e5
:109298006080780080407800d0d92000000041002c
:1092a800014878002e009000810420008e80400044
:1092b8000000400060807800e8004700801f7800c8
:1092c80090a72a00801f7800010078006ae907004b
:1092d800e4875700680047006d0c07002e009000d7
:1092e8000000e80020079800ae0090003e009000c3
:1092f800808f5000d3ff3400f0a72a00640c0700c9
:109308000080fa00000006000c00fa00889fbe00ea
:1093180040079800510798004e0090001000be00ca
:109328000004be005e0090000000e800cf80de0070
:10933800b1e107000001be00000020000112240076
:10934800ece207000001be000800be00b5e207001d
:10935800008fbe004e0090001000be006011b800e3
:1093680030e207000000e000010035000600370089
:109378001e00be0002002000030a2400c9e1070005
:10938800008fbe00050037001e00be00020020004e
:10939800030a2400c4e10700008fbe001e00be00bf
:1093a80002002000031224005ce20700008fbe00c8
:1093b8001e00be0064014700b1e307002e009000c4
:1093c800be0090000004be005e009000cf80de006a
:1093d80089e107000001be000000200001122400fe
:1093e800c4e207000001be000800be004be207000f
:1093f8004f04be000080fa00000006006000fa007a
:10940800889fbe008a9fbe0060c798000040eb009e
:10941800004f78006ec090000080fb006101b90029
:1094280000fd2f00f1ff2f0002014000838148005a
:10943800622f9800732f9800c003200001002000bd
:109448006e299000fe299000800f5100818f5900ed
:10945800c5043e006e289000fe28900000600100c0
:109468003c003700580037008a00370008013700f1
:109478008001370099013700b2013700cb0137006e
:10948800e401370020023700b7043700b60437007c
:10949800b5043700b4043700b3043700b20437000a
:1094a800b104370099033700b7033700c403370006
:1094b8004e043700520437005c043700a704370015
:1094c80052023700a8043700a7043700a604370063
:1094d800a5043700a4043700a3043700a20437000a
:1094e800a1043700a00437009f0437009e0437000a
:1094f8009d0437009c0437009b0437009a0437000a
:109508009904370098043700970437009604370009
:109518009504370094043700930437009204370009
:10952800910437001d023700310237006e02370000
:1095380099023700ae023700cc023700e10237004b
:1095480089043700e202370089043700e302370054
:10955800e50237000040eb0005eeb700a4fd070068
:10956800200798002e009000e10f40008004320090
:10957800ae009000803e2000808f50000d003c001f
:109588002e009000e90f50000a0034002e009000d1
:10959800cf80de0018e1070002002000832c2400a1
:1095a800dee10700506e8800616e88004a070700f8
:1095b8000200370040a82a00b50b070010c0b3000e
:1095c80005eeb7006a0437000040eb0005eeb7006f
:1095d80087fd070020079800226e8000007d20008c
:1095e800110009000200d800806e8800806e80009b
:1095f800f00f50000200340000012000806e880047
:10960800816e80002e009000808f5000140035007d
:109618002e0090000000e00011003400ae00900021
:10962800716e8800706e8000800078002000200035
:1096380076080700706e8000e6004700801f7800fb
:10964800a0aa2a00801f7800010078008ae8070095
:10965800e4875700660047008d0b07000a003700b3
:10966800806e8000e6004700801f7800c0ad2a00a9
:10967800801f7800010078007fe80700e487570022
:1096880066004700820b070010c0b30005eeb70064
:10969800370437000040eb0005eeb70054fd070023
:1096a80020079800ae009000706b8000808f5000fb
:1096b8006a003e002e0090000000e00067003500c0
:1096c8002e009000506b8800506b8000e600470029
:1096d800801f780080b22a00801f7800010078007f
:1096e80065e80700e487570066004700680b070035
:1096f800516b8000606b8000808f50001300360033
:10970800506b800000004000606b8800616b800037
:10971800706b8000808f500002003600706b8000f4
:10972800606b8800506b8000e6004700801f78005f
:1097380030b52a00801f7800010078004ee8070045
:10974800e487570066004700510b0700506b800004
:1097580000004000000478006140b900a6e007005e
:10976800402f9800512f98000800e00007003d00a6
:1097780002002000037824004e289000de28900084
:10978800c9e00700402f9800512f9800926e800082
:10979800a36e80004e289000de2890005fe107004d
:1097a80002002000832c24009ee1070040e107000e
:1097b800806b8800616b8000506b800000805000d7
:1097c80000004000000478006140b9008ae007000a
:1097d800202f9800312f98000800e00007003d0076
:1097e80002002000037824002e289000be28900054
:1097f800ade00700202f9800312f9800926e80006e
:10980800a36e80002e289000be28900043e1070038
:1098180002002000832c240082e1070024e10700d5
:10982800906b880010c0b300e0edb700401f200027
:10983800a06b8800d0cc2c00c1dc2300e06e88002f
:10984800f16e8800806b800038090700906b8000fb
:109858006009070047fd07000a003700706b8000a9
:10986800e6004700801f780080b92a00801f780032
:109878000100780000e80700e48757006600470009
:10988800030b070010c0b30005eeb700b80337009c
:109898000040eb0005eeb700d5fc07002007980054
:1098a800ae009000706b8000808f500064003e0016
:1098b8002e0090000000e000610035002e009000ae
:1098c800606b8800606b8000e6004700801f7800ae
:1098d800b0bb2a00801f780001007800e6e7070087
:1098e800e487570066004700e90a0700516b8000cb
:1098f800606b8000808f50000d003600606b800028
:109908000000d100506b8800506b8000e6004700d3
:10991800801f780060be2a00801f78000100780050
:10992800d5e70700e487570066004700d80a070014
:10993800506b800000004000000478006140b900ce
:109948002de00700002f9800112f98000800e00074
:1099580007003d0002002000037824000e28900034
:109968009e28900050e00700002f9800112f9800c3
:10997800926e8000a36e80000e2890009e289000b2
:10998800e6e0070002002000832c240025e1070000
:10999800c7e00700806b8800616b8000506b800017
:1099a8000080500000004000000478006140b900c9
:1099b80011e0070060279800712798000800e00070
:1099c80007003d0002002000037824006e2090006c
:1099d800fe20900034e00700602798007127980067
:1099e800926e8000a36e80006e209000fe20900092
:1099f800cae0070002002000832c240009e10700c8
:109a0800abe00700906b880010c0b300e0edb70032
:109a1800401f2000a06b8800d0cc2c00c1dc2300a4
:109a2800e06e8800f16e8800806b8000bf08070038
:109a3800906b8000e7080700cefc07000a0037009b
:109a4800706b8000e6004700801f7800e0c22a00a3
:109a5800801f78000100780087e70700e487570037
:109a6800660047008a0a070010c0b30005eeb70079
:109a78003f0337005efc070020079800ae00900007
:109a8800f00f2000808f500011003c002e00900045
:109a98000000e0000e0035002e009000faedb7003f
:109aa800b4fc0700e60047002e019000821f7800f2
:109ab80010c52a00801f7800010078006ee70700b3
:109ac800e487570066004700710a0700280337003b
:109ad80020c72a006e0a07002503370044fc070048
:109ae80020079800ae009000f00f2000808f5000f3
:109af80011003c002e0090000000e0000e00350030
:109b08002e009000fcedb7009afc0700e600470025
:109b1800ae019000831f780020c92a00801f7800ba
:109b28000100780054e70700e48757006600470003
:109b3800570a07000e03370090cb2a00540a070083
:109b48000b0337002afc070020079800ae0090009e
:109b5800f00f2000808f500011003c002e00900074
:109b68000000e0000e0035002e009000fbedb7006d
:109b780080fc0700e60047002e009000801f780058
:109b8800f0cd2a00801f7800010078003ae707002e
:109b9800e4875700660047003d0a0700f4023700d3
:109ba80000d02a003a0a0700f102370010fc07002b
:109bb80020079800ae009000f00f2000808f500022
:109bc80011003c002e0090000000e0000e0035005f
:109bd8002e009000fdedb70066fc0700e600470088
:109be8002e019000821f780020c92a00801f78006b
:109bf8000100780020e70700e48757006600470067
:109c0800230a0700da02370090cb2a00200a07004f
:109c1800d70237000040eb0005eeb700f4fb070061
:109c280020079800ae009000007d2000808f500033
:109c380032003c002e0090000000e0002f003400ad
:109c4800ae019000236e8800226e8000007d200007
:109c5800110009000200d800806e8800806e800024
:109c6800f00f50000200340000012000806e8800d0
:109c7800816e8000706e8000808f500010003d0063
:109c8800806e8000706e8800706e800080007800a2
:109c980020002000dd060700706e8000e600470007
:109ca800801f7800b09a2a00801f78000100780091
:109cb800f1e60700e487570066004700f40907004b
:109cc800206e8000fa0a0700206e8000e600470038
:109cd800801f7800409d2a00801f780001007800ce
:109ce800e5e60700e487570066004700e809070033
:109cf80010c0b30005eeb7009d023700409f2a0050
:109d0800e30907009a0237000040eb0005eeb700b0
:109d1800b7fb070020079800ae009000e00f200076
:109d2800808f50001a003c002e0090000000e000d8
:109d3800170034002e009000b06e8800b16e8000cd
:109d4800800c20000088b900c06e8800c06e8000ba
:109d58008000780030002000ac060700c06e80004c
:109d6800e6004700801f780000d22a00801f780094
:109d780001007800c0e60700e48757006600470046
:109d8800c309070010c0b30005eeb700780237001a
:109d980080d42a00be090700750237001100200090
:109da8008000200099060700000000000000000065
:109db800000000000000000000000000000000009b
:109dc80000000000000000000040eb00efedb700cd
:109dd80021002000800020008c06070010002000d1
:109de800e0688800f0d62a00a90907006002370059
:109df8000000eb00e06888008000eb008000200095
:109e08008206070070d82a00a1090700f0d92a00a5
:109e18009f09070010db2a009d090700e0dc2a00e3
:109e28009b09070050de2a009909070010e02a0064
:109e380097090700d0e12a009509070030e32a00b6
:109e48009309070080e42a0091090700e0e52a0049
:109e58008f09070030e72a008d09070040e82a002b
:109e68008b090700a0e92a008909070040ec2a00ad
:109e78008709070030ef2a008509070010f12a003a
:109e88008309070040f32a008109070090f52a009a
:109e98007f09070070f72a007d090700c0f92a002a
:109ea8007b090700f0fa2a007909070050fc2a000c
:109eb80077090700b0fd2a007509070030ff2a005e
:109ec8007309070070012b0071090700d0022b00ed
:109ed8006f09070040042b006d090700c0052b001f
:109ee8006b090700220237000040eb0005eeb700bf
:109ef8003ffb0700200798002e009000e10f50005c
:109f080010003a00906f80000000e00003003a0063
:109f180050062b005e0907000a00370010002000d9
:109f2800a06f8800c5a2a900c1a2a900a06f8000e7
:109f3800800078007000200034060700200b2b00fa
:109f4800530907002e0090000000e0000a003a00c4
:109f58000000eb00a06f8800c5a2a800c1a2a9005c
:109f6800a06f80008000780070002000270607009e
:109f7800f00d2b00460907002e009000e10f50005d
:109f880002003400c0102b004109070010c0b300c4
:109f980005eeb700f601370015fb0700200798000b
:109fa8002e0090000000e00004003a000040eb00a2
:109fb800f6edb70070132b00350907002e0090004e
:109fc800e10f500004003a0010c0b300f6edb700ee
:109fd80010182b002e0907002e009000e10f5000ea
:109fe800e3013400b01c2b0029090700e001370009
:109ff800fffa0700200798002e0090000000e000fc
:10a0080017003400ae009000f0702200808f5000de
:10a0180013003c002e009000823e20001100090031
:10a028000200d800cf80de0073de0700906e880043
:10a03800a16e8800e60047002e019000821f78007c
:10a04800a0232b00801f7800010078000ae6070093
:10a05800e4875700660047000d090700c401370070
:10a0680050262b000a090700c1013700e0fa070053
:10a07800200798002e0090000000e00004003a003d
:10a088000040eb00f8edb70040292b00000907005d
:10a098002e009000e10f500004003a0010c0b300f9
:10a0a800f8edb700d02a2b00f90807002e00900021
:10a0b800e10f5000ae013400602c2b00f4080700bb
:10a0c800ab01370010002000e8fb0700a8013700ab
:10a0d80020002000e5fb0700a501370090c0b30071
:10a0e800c6fc0700a2013700506e8000616e800038
:10a0f80066014700809fbe00a02e2b00801f7800bd
:10a1080002007800dce50700e68757006600470094
:10a11800df080700706e8000e6004700801f7800a7
:10a1280060302b00801f780001007800d2e507001e
:10a13800e487570066004700d5080700606b800079
:10a14800516b800066014700801f7800811f7800ee
:10a1580050312b00801f780002007800c6e5070008
:10a16800e687570066004700c9080700fccdbf0016
:10a178008080fb00facdbf000080fb00660147002d
:10a18800811f7800801f7800f0322b00801f780034
:10a1980002007800b8e50700e68757006600470028
:10a1a800bb080700fdcdbf008080fb00fbcdbf00d2
:10a1b8000080fb0066014700811f7800801f78003f
:10a1c800d0342b00801f780002007800aae5070031
:10a1d800e687570066004700ad080700206e80003c
:10a1e800e6004700801f7800b0362b00801f7800fb
:10a1f80001007800a0e50700e487570066004700e3
:10a20800a3080700a06f8000e6004700801f7800c1
:10a2180080372b00801f78000100780096e5070042
:10a22800e48757006600470099080700f6cdbf008d
:10a238000000fb00e6004700801f7800e0382b0094
:10a24800801f7800010078008be50700e48757003d
:10a25800660047008e080700f8cdbf000080fb00ad
:10a26800e6004700801f7800a03a2b00801f780086
:10a278000100780080e50700e48757006600470082
:10a2880083080700626f8000efcdbf008080fb006d
:10a29800eecdbf000080fb00e6014700821f78007a
:10a2a800811f7800801f7800603c2b00801f780099
:10a2b8000300780070e50700e8875700660047004c
:10a2c80073080700106f8000216f8000d26e800035
:10a2d80003708000946b8000e6024700809fbe00f8
:10a2e800821f7800831f7800841f7800703f2b003e
:10a2f800801f7800050078005fe50700ec875700ad
:10a308006600470062080700190137000040eb00ab
:10a3180005eeb70010432b005d08070060492b00cd
:10a328005b0807000000eb001007980010003700da
:10a338001e009000da040700e6004700801f78003e
:10a348009e019000831f7800904c2b00801f78009e
:10a358000100780048e50700e687570066004700d7
:10a368004b0807001e0090000000e8001007980046
:10a378001e009000ef0f5000edff340010c0b30036
:10a3880005eeb700fa00370019fa070002eeb70029
:10a3980002cebf000080fb00e6004700801f780067
:10a3a800004e2b00801f78000100780032e507007e
:10a3b800e48757006600470035080700ec003700bf
:10a3c8000bfa070020079800a0002000810607006c
:10a3d8002e0090000000e000030032002e009000e4
:10a3e800e20f500027003a00904f2b002808070082
:10a3f8000000eb00100798001f003700a4030700b7
:10a40800a0002000a604070000057800e000200056
:10a41800a304070080057800d0002000a0040700ee
:10a4280000047800c00020009d0407008004780024
:10a43800b00020009a040700e60047008a1f780051
:10a448008b1f7800881f7800891f7800801f78008c
:10a45800f0502b00801f78000100780006e5070007
:10a46800ec87570066004700090807001e009000a7
:10a478000000e800100798001e009000e10f50004f
:10a48800deff34002e009000e10f50000300320080
:10a498002e009000e20f500027003a0040542b0095
:10a4a800fb0707000000eb00100798001f003700ab
:10a4b8005d030700a000200079040700000578006c
:10a4c800e00020007604070080057800d000200016
:10a4d8007304070000047800c0002000700407001f
:10a4e80080047800b00020006d040700e6004700f3
:10a4f8008a1f78008b1f7800881f7800891f7800d2
:10a50800801f7800f0502b00801f78000100780031
:10a51800d9e40700ec87570066004700dc0707000e
:10a528001e0090000000e800100798001e00900030
:10a53800f30f5000deff3400906b80002506070003
:10a548002e009000e30f500089003a00110020000f
:10a5580080002000ad04070000000000000000009b
:10a5680000000000000000008000eb0080002000d8
:10a57800a6040700a0552b00c5070700a00020006f
:10a588004704070000057800e000200044040700a5
:10a5980080057800d00020004104070000047800fe
:10a5a800c00020003e04070080047800b0002000ae
:10a5b8003b040700e60047008a1f78008b1f7800dd
:10a5c800881f7800891f7800801f7800f0502b00c2
:10a5d800801f780001007800a7e40700ec87570087
:10a5e80066004700aa0707006100370080f90700e6
:10a5f800200798002e009000007088005c0037004b
:10a60800306e8000e6004700801f780040572b001e
:10a61800801f78000100780097e40700e48757005e
:10a62800660047009a0707005100370070f90700d5
:10a6380020079800ae00900040062000808f500050
:10a6480043003400ae009000703e2000808f500020
:10a658003f003c00ae009000a16b880010c0b30022
:10a66800e0edb700916b8000d06e800000017800ab
:10a67800110009008280d800000478006140b90008
:10a68800dddc070040279800512798000800e0000b
:10a6980007003d0002002000037824004e209000af
:10a6a800de20900000dd0700402798005127980021
:10a6b8004e219000de219000126f8800236f8800e1
:10a6c800186f8000296f8000a06b8000cf80de00ab
:10a6d800c9dc07000001be000800be008fdd0700ce
:10a6e800106f8800216f8800106f8000216f800034
:10a6f8000200200003f823004add07000000e00004
:10a7080001003500040037000000200001f8230094
:10a71800106f8800216f8800106f8000216f800003
:10a7280066014700809fbe00ae019000831f78003d
:10a73800005a2b00801f7800020078004ee40700c2
:10a74800e8875700660047005107070008003700f0
:10a75800b05c2b004e070700050037000040eb00f7
:10a76800e0edb70002003700f05e2b004807070055
:10a778001e80fb004f05be004f04be000080fa009b
:10a78800000006000200fa000040eb00e2060700a5
:10a798000000e000fcff320000c0eb00de0607000e
:10a7a8000000e000fcff320010c0b300da0607002a
:10a7b8000000e000fcff320000c0eb00d6060700f6
:10a7c8000000e000fcff320020c0b300d206070002
:10a7d8000000e000fcff3200506e8000616e8000d7
:10a7e80002002000031224008edd070030dd070080
:10a7f800c90607000000e000f7ff3200206e800065
:10a80800a2002000110009000200d800c2060700bb
:10a818000000e000f9ff3200706e8000be060700fd
:10a828000000e000fcff3200506b8000ba06070011
:10a838000000e000fcff3200606b8000b6060700f5
:10a848000000e000fcff3200d06e8000b206070076
:10a858000000e000fcff3200906b80004800de0042
:10a868000040e800ac0607000000e000faff3200f4
:10a87800906b80000040e800a70607000000e00099
:10a88800fbff3200a06b80004880de000040e8003b
:10a89800a10607000000e000faff3200a06b80006c
:10a8a8000040e8009c0607000000e000fbff3200c3
:10a8b800e0cdbf000040e800970607000000e00078
:10a8c800fbff3200f8cdbf000040e8009206070009
:10a8d8000000e000fbff3200e06880000040e80074
:10a8e8008d0607000000e000fbff3200facdbf0034
:10a8f800890607000000e000fcff3200fccdbf0025
:10a90800850607000000e000fcff32000000eb00b5
:10a91800000f7800090037009e00780090d82000ca
:10a9280000804000104078000040e8007a060700e8
:10a938000000e000f8ff32001e0fe800f9cdbf006c
:10a948000080fb009e0f5000f3ff3c000080fa00df
:10a95800000006004200fa00889fbe008a9fbe00e1
:10a968008c1f7800e2688000f8cdbf008081fb0072
:10a97800e0cdbf000082fb00a56b8000966b8000d5
:10a98800d76e8000686b8000596b80007a6e8000fb
:10a998002b6e8000506e8000616e80000e86e8008d
:10a9a800821f7800831f7800841f7800851f780035
:10a9b800861f7800871f7800881f7800891f780015
:10a9c8008a1f78008b1f7800809fbe0000602b00d4
:10a9d800801f78000c007800a7e30700fa8757006b
:10a9e8000e80e800aa060700fccdbf008080fb00af
:10a9f800facdbf000080fb000e81e800811f7800bf
:10aa0800801f780090622b00801f78000200780079
:10aa180099e30700e68757000e80e8009c060700c8
:10aa28000000eb00000f78000f0037009e00780050
:10aa380090d8200000804000104078000080fb0083
:10aa48008e80e800801f780030632b00801f78001c
:10aa58000100780088e30700e48757000e80e800cb
:10aa68008b0607001e0fe800f9cdbf000080fb0031
:10aa78009e0f5000edff3c0070632b00840607001a
:10aa88004f0678004f05be004f04be000080fa0054
:10aa9800000006004200fa00307280000000e0006a
:10aaa8002d0032000000eb0030728800e8c2bf00c1
:10aab8000080fb000000d100614060000004a2009b
:10aac800614060006140600000414000812e20002c
:10aad80091407800d0cfb30000c060000240700001
:10aae800e8e2b700e422a900c16d8000805121008e
:10aaf800808f5000020034000000eb00c06d880019
:10ab0800f6cdbf000004e00008003a00e0688000cd
:10ab1800e10f500003003a0010c0b300f7edb70092
:10ab28000d0037008bff07000b003700e06880003e
:10ab3800e10f500003003a0010c0b300f7edb70072
:10ab4800050037000040eb00f30507000000e000b7
:10ab5800fcff32000bff07000080fa00000006002f
:10ab68000400fa0002cebf000004e0002600320014
:10ab780002cebf00e14f50000300320002cebf00fa
:10ab8800e34f500004003a0031e020009140780083
:10ab980010c0b3008b01070002cebf00e24f500087
:10aba8000300320002cebf00e34f500004003a0019
:10abb80041e020009140780020c0b30081010700e7
:10abc800e922a800e522a90003cebf000040e80062
:10abd80003eeb70004cebf000040e90004eeb70062
:10abe80003cebf00e14f400002003a000040eb00f6
:10abf80003eeb70004cebf000004e00002003a00f4
:10ac080000c0eb0004eeb700ffcdbf000004e00079
:10ac180037003a00e0688000e10f500034003a0045
:10ac2800d702a800d302a90000000000000000001d
:10ac3800000000000000000000000000000000000c
:10ac48000000000000000000d702a900d302a900fc
:10ac58000000eb0010079800170037009e009000d6
:10ac680090d82000008040009040780010c0b300c9
:10ac7800540107009e009000d0d9200000804000b9
:10ac88009040780020c0b3004e0107000000eb00a0
:10ac9800000f780002003700000000001e0fe800d7
:10aca800007080009e0f1000fbff35001e00900012
:10acb8000000e80010079800f9cdbf008080fb0075
:10acc8001e009000808f5000e4ff3c0081c0b3005c
:10acd80010c0b3003b01070081c0b30020c0b3001f
:10ace8003801070010c0b300ffedb70001003700be
:10acf800020007000080fa00000006005200fa0077
:10ad0800889fbe008a9fbe006000b800008fbe000a
:10ad1800e0688000e10f500026013a00f8cdbf003e
:10ad2800e14f500023013a000000eb00e068880082
:10ad3800a00020005a020700eeedb700eecdbf00dc
:10ad480063406000eeedb700eecdbf00e24f50006b
:10ad580014013a00efcdbf000004e0000300320008
:10ad6800efcdbf00e34f50000e013a008000eb002a
:10ad780080002000a502070010002000606f8800f6
:10ad8800e802a800e402a900f8cdbf00e14f500096
:10ad980016003a00f6cdbf000004e00009003a00b2
:10ada800f7cdbf00e14f500003003a00e9fe07006d
:10adb8000040eb00f7edb700b0632b00b4050700c7
:10adc8000a003700f7cdbf00e14f500003003a00fa
:10add8006cfe07000040eb00f7edb7000040eb0009
:10ade8004d0507000000e000fcff32000000eb000a
:10adf800606f88006000b800106c8800216c8800c3
:10ae08000000eb00406f88000040eb00eaedb7005f
:10ae18006000b800f06b8800016c88000000eb004f
:10ae28003007980005003700ff00070088edb700dd
:10ae38003e0090000000e800300798003e009000b7
:10ae4800fd0f5000f8ff34000000eb0030079800b9
:10ae5800a4003700f400070088edb700606f800099
:10ae68000000e800606f88000040eb00e6edb700e6
:10ae7800e0cdbf00e14f500042003a00106f800063
:10ae8800216f80000041eb0002d7980002002000eb
:10ae980003f8230008dd07000000e00001003a0085
:10aea8000200370010c0b30000d798000ed0900001
:10aeb8000004a2000004e00032003a00f06b8000b9
:10aec800016c80000200200003f82300f6da070076
:10aed800f06b8800016c880088d82000184478003e
:10aee8000800fb00cf80de00c3da07006027980067
:10aef800712798000804e00007003d0002002000c8
:10af0800033824006e209000fe209000e6da070047
:10af180060279800712798006e219000fe2190000c
:10af28001e00be00e0da0700008fbe00106f800030
:10af3800216f8000f26b8000036c800039db070012
:10af48000000e000010035003c00370010c0b300ed
:10af5800e6edb700f26b8000036c80001e00be00b7
:10af68006edb070031db0700306c88006000b8003a
:10af7800008fbe006000b800f06b8800016c88008c
:10af88002e00370010c0b300e6edb700d06b80008c
:10af9800e16b8000e26e8000f36e8000a1db0700a9
:10afa8000005be0088cdbf000080fb00cf80de001a
:10afb80091da07000004be00e26e8000f36e8000a4
:10afc8000000200001f82300b6da07000001be00e7
:10afd8000800be0093db07000001be000a00be00a7
:10afe800b1da070011db0700306c880088d8200030
:10aff800184478000800fb00cf80de007eda0700e6
:10b0080040279800512798000804e00007003d00f9
:10b0180002002000033824004e209000de2090001b
:10b02800a1da070040279800512798004e20900089
:10b03800de209000d06b8800e16b8800f8cdbf005f
:10b04800e14f500024003a00e6cdbf00e14f500028
:10b0580021003a00f6cdbf000004e0000b003a00e2
:10b06800306c8000e8004700801f780030632b00b8
:10b07800801f780001007800ffe10700e48757008f
:10b08800680047000205070009003700306c80009f
:10b098000000e00002003a0010002000306c880038
:10b0a800306c80009c0407000000e000fcff3200c8
:10b0b800406f80000000e800406f8800306c80001e
:10b0c80080407800eacdbf0000c04000eaedb7003c
:10b0d8000000eb00306c88003e0090000000e800a3
:10b0e80030079800be019000916b8000d06e800000
:10b0f80000017800110009008280d8007e0050000d
:10b10800808f510053ff3900e802a900e402a9002a
:10b11800f8cdbf00e14f500010003a00f6cdbf0057
:10b128000004e0000d003a00eacdbf000080fb00fb
:10b13800416f800068014700801f7800811f7800f8
:10b14800d0632b00801f780002007800cae1070056
:10b15800e687570068004700cd040700110020006b
:10b1680080002000a9010700000000000000000086
:10b1780000000000000000000000000000000000c7
:10b1880000000000000000000000000000000000b7
:10b1980000000000000000002100200080002000c6
:10b1a8009a010700eecdbf00efedb70010002000b8
:10b1b800e06888004f05be004f04be000080fa001a
:10b1c800000006000400fa00204798003147980064
:10b1d80005cebf00e14f500011003a00e922a90056
:10b1e800e522a9002e409000e14f500003003a00ec
:10b1f800c5c2a900c1c2a90002003700c5c2a80083
:10b20800c1c2a9003e4090000080fb00b016880033
:10b21800e902a900e502a900e902a800e502a900df
:10b228000080fa00000006000200fa00d7a2a80079
:10b23800d3a2a90001168000f00f20000080700042
:10b2480000168800d782a900d382a900d762a80077
:10b25800d362a90000000000000000000000000008
:10b2680000000000d782a800d382a90000000000d7
:10b27800000000000000000010168000000f780099
:10b288001e0078000080fb000080fa000000060025
:10b298000200fa00110020000000eb005b0107002b
:10b2a800d762a800d362a900d7a2a900d3a2a90097
:10b2b8000000000010168000000f7800d7a2a80038
:10b2c800d3a2a9008000eb000000eb004f010700ab
:10b2d8000080fa00000006005000fa00889fbe00b7
:10b2e80010002000d06e8800506e8000616e8000d3
:10b2f80002002000030a24004ada07000000e000e8
:10b30800010035000200370020002000d06e8800c0
:10b31800506e8000616e800002002000030224004d
:10b3280040da07000000e0000100350002003700a5
:10b3380040002000d06e8800506e8000616e800052
:10b348006266260063fa230036da07000000e00090
:10b35800010035000200370080002000d06e880010
:10b36800526e8000636e800000002000813424004b
:10b378006ada07002dda0700406b8800526e8000f9
:10b38800636e800000002000813c240063da07001f
:10b3980047da0700706b8800706b80000000d100ee
:10b3a800606b8800606b80000000d100506b8800e3
:10b3b800506b800000004000000478006140b90034
:10b3c8008dd9070060279800712798000800e000d1
:10b3d80007003d0002002000037824006e20900042
:10b3e800fe209000b0d907006027980071279800c8
:10b3f800926e8000a36e80006e209000fe20900068
:10b4080046da070002002000832c240085da0700b2
:10b4180027da0700806b8800616b8000506b800022
:10b428000080500000004000000478006140b9002e
:10b4380071d9070040279800512798000800e000bc
:10b4480007003d0002002000037824004e209000f1
:10b45800de20900094d907004027980051279800d3
:10b46800926e8000a36e80004e209000de20900037
:10b478002ada070002002000832c240069da07007a
:10b488000bda0700906b880010c0b300e0edb7003e
:10b49800401f2000a06b8800916b8000a06b80008b
:10b4a80000017800110009008280d800800078002f
:10b4b800d06e800000017800110009008280d80059
:10b4c800000478006140b9004bd907002027980094
:10b4d800312798000800e00007003d000200200026
:10b4e800037824002e209000be2090006ed907001b
:10b4f80020279800312798002e209000be20900029
:10b50800106f8800216f8800106f8000216f800005
:10b518000200200003f82300c2d907000000e00061
:10b5280001003500040037000000200001f8230066
:10b53800106f8800216f8800806b8000fb01070076
:10b54800906b800023020700d06e80008000780096
:10b55800f0002000ad000700506e8000616e800092
:10b56800809fbe0070642b00801f78000e0078005a
:10b57800c1e00700e68757000e007800c403070003
:10b58800606b8000801f7800d0662b00801f7800d9
:10b598000e007800b8e00700e48757000e00780036
:10b5a800bb030700506b8000801f7800d0682b0019
:10b5b800801f78000e007800afe00700e48757008e
:10b5c8000e007800b2030700406b8000800078000e
:10b5d800100020008d000700606b80000000400014
:10b5e800000478006140b90003d9070000279800db
:10b5f800112798000800e00007003d000200200025
:10b60800037824000e2090009e20900026d9070081
:10b618000027980011279800926e8000a36e800082
:10b628000e2090009e209000bcd907000004be00a8
:10b63800f9cdbf000080fb00cf80de00eed8070008
:10b648006266260063002c00f6d907000001be00e0
:10b658000800be0014d907000004be00f9cdbf00e1
:10b668000080fb00cf80de00e3d80700a299290004
:10b6780093e12300ebd907000001be000800be00db
:10b68800a6d9070069d9070000708800b9f5070036
:10b69800b8f507004f04be000080fa00000006005d
:10b6a8000600fa0020079800ae009000f00f200076
:10b6b8000080600020079800e016800010079800be
:10b6c8009e00900000f02f00808060002e00900007
:10b6d80000807000100798001e009000e016880097
:10b6e800c116800000f02f0000806000c01688009e
:10b6f800d7a2a800d3a2a90001168000f00f20004d
:10b708000080700000168800d782a900d382a900a3
:10b71800d762a900d3a2a900000000000000000021
:10b728000000000000000000000000000000000011
:10b73800000000000000000010168000000f7800d4
:10b7480000000000000000000000000000000000f1
:10b75800d782a800d382a900d762a800d362a90023
:10b7680000000000000000000000000000000000d1
:10b77800d7a2a900d3a2a900f00f20001e0f6000d5
:10b788001e0078000080fa00000006000400fa009d
:10b7980001168000f00f200000807000001688005d
:10b7a800d7a2a800d3a2a900d782a800d382a90053
:10b7b800d762a800d362a9000000000000000000c2
:10b7c800000000000000000010168000000f780044
:10b7d8000000000000000000000000000000000061
:10b7e8000000000000000000000000000000000051
:10b7f800d7a2a900d3a2a900f00f20001e0f600055
:10b808001e0078000080fa00000006004a00fa00d6
:10b818002027980031279800ae209000f00f2000d4
:10b828000080600020279800be209000f00f2000c4
:10b838000080600030279800d7a2a900d3a2a900f1
:10b84800d762a800d362a900e0168000100798000c
:10b858009e00900000f02f00808060002e20900055
:10b8680000807000100798001e009000e016880005
:10b87800c116800000f02f0000806000c01688000c
:10b8880020168000100798009e00900000f02f00fe
:10b89800808060003e2090000080700010079800b3
:10b8a8001e009000201688000116800000f02f006e
:10b8b8000080600000168800d7a2a800d3a2a900c3
:10b8c800d762a900d3a2a900000000000000000070
:10b8d8000000000000000000d7a2a900d3a2a90020
:10b8e8000000000000000000000000000000000050
:10b8f8000000000000000000000000000000000040
:10b90800d762a800d362a900000000000000000070
:10b9180000000000000000002e20900060ff0700db
:10b92800000f78000000eb00402798003e209000b0
:10b938009e0f100002003a001000200040279800d7
:10b948004e2090000080fa00000006000600fa0071
:10b95800000f780011079800400020009e0f10008b
:10b9680003003e001e009000ff0f50000300360049
:10b978000000eb0020079800040037009e009000ac
:10b988001e007800a1ff0700200798002e009000f5
:10b998000080fa00000006000400fa00000f78009a
:10b9a800f00f20009e0f1000030036000000eb008f
:10b9b80010079800040037009e007800500020000f
:10b9c80092ff0700100798001e0090000080fa0000
:10b9d800000006005400fa0010002000000f780054
:10b9e800e06a2b00aa020700300020001007980028
:10b9f8008a0037001e00e000080032001100200015
:10ba08001e00900081ff07000000e00003003200e4
:10ba180010002000102f9800020037008000eb0073
:10ba2800112f98001e289000000f78001e00e000db
:10ba380008003200210020001e00900073ff07005c
:10ba48000000e0000300320011002000012f9800e0
:10ba5800020037000000eb00002f98008e289000ad
:10ba6800010f78001e00e0000800320041002000ad
:10ba78001e00900065ff07000000e0000300320090
:10ba88001000200070279800020037008000eb00ab
:10ba9800712798007e209000000f78001e00e000bb
:10baa80008003200810020001e00900057ff0700a8
:10bab8000000e00003003200110020006127980018
:10bac800020037000000eb0060279800ee2090008d
:10bad800010f78001e00e00008003200010120007c
:10bae8001e00900049ff07000000e000030032003c
:10baf8001000200050279800020037008000eb005b
:10bb0800512798005e209000000f78001e00e0008a
:10bb180008003200010220001e0090003bff0700d1
:10bb28000000e000030032001100200041279800c7
:10bb3800020037000000eb0040279800ce2090005c
:10bb4800010f78001e00e000080032000104200008
:10bb58001e0090002dff07000000e00003003200e7
:10bb68001000200030279800020037008000eb000a
:10bb7800312798003e209000000f78001e00e0005a
:10bb880008003200010820001e0090001fff070077
:10bb98000000e00003003200110020002127980077
:10bba800020037000000eb0020279800ae2090002c
:10bbb800010f78001e00e0000a003a006400470008
:10bbc8009e009000811f7800a16c2b00811f7800d7
:10bbd80029df0700e4875700640047002c020700ac
:10bbe80009003700640047009e009000811f78001c
:10bbf800f16d2b00811f78001fdf0700e4875700d5
:10bc0800640047002202070010002000000f78009f
:10bc18001e0090000000e800100798001e00900029
:10bc2800e60f500073ff36001e0078000080fa000f
:10bc3800000006000600fa00606f2b0014020700df
:10bc480080702b001202070090712b001002070071
:10bc5800d762a800d362a900d782a800d382a9001e
:10bc6800d7a2a800d3a2a9002ac3a8002ae3a80043
:10bc78000000eb00000f7800020037000000000011
:10bc88001e0fe800300620009e0f1000fbff360054
:10bc980050ff07000000e00020003200d0722b00a7
:10bca800fb010700406e8000800078000000eb0078
:10bcb800d6fe0700406b800080007800100020004e
:10bcc800d2fe0700706e80008000780020002000ff
:10bcd800cefe0700c06e8000800078003000200093
:10bce800cafe0700806b800010000700906b800080
:10bcf80038000700a06f80008000780070002000e6
:10bd0800c2fe0700816f800080002000bffe070090
:10bd1800a0732b00de0107000200370030752b00ee
:10bd2800db0107000080fa00000006000800fa00a6
:10bd38001007980010002000000f78001e00e00097
:10bd48000a0032009e009000f00f20008080600002
:10bd580090002000adfe07000000e0000300320064
:10bd68001000200030079800020037000000eb00a8
:10bd7800300798003e009000000f78001e009000e9
:10bd88004880de00100798001e00e0000a0032001c
:10bd98009e009000f00f200080806000400020008e
:10bda8009afe07000000e0000300320010002000a7
:10bdb80020079800020037000000eb0020079800d9
:10bdc8002e009000000f78001e0078000080fa0016
:10bdd800000006004a00fa00202798001000200002
:10bde800000f78001e00e0000a003200ae2090002c
:10bdf800f00f2000808060006000200083fe0700b4
:10be08000000e000030032001000200040279800e6
:10be1800020037000000eb00402798004e209000f9
:10be2800000f78002e2090004880de001007980050
:10be38001e00e000080032009e0090005000200024
:10be480072fe07000000e00003003200100020002e
:10be580030279800020037000000eb0030279800d8
:10be68003e209000000f78001e0078000080fa0045
:10be7800000006000200fa000000eb00000f780046
:10be880002003700000000001e0fe80090002000ac
:10be98009e0f1000fbff34000080fa00000006002f
:10bea800809fbe000000fa00206880000000e000cb
:10beb80010003200116880000080200000804000df
:10bec800104078000080fb00201188000100e80085
:10bed8001068880011688000f01f20000080600052
:10bee80010688800206880000000e9002068880049
:10bef800010037009580a9008580a9000080fa001c
:10bf08004f00be0000400600809fbe000000fa00ff
:10bf1800506880000000e000100032004168800096
:10bf280000a0200000804000104078000080fb0046
:10bf3800a01188000100e80040688800416880007e
:10bf4800f01f200000806000406888005068800072
:10bf58000000e900506888000100370097e0a90058
:10bf680087e0a9000080fa004f00be0000400600ec
:10bf7800809fbe000200fa000000370022c2bf0006
:10bf8800644060000004e0000300320030118000cb
:10bf9800004f7800f9ff370022c2bf0062406000fe
:10bfa8000004e000020032002222a9001800370035
:10bfb80022c2bf00614060000004e00014003200ab
:10bfc80030118000004f780081688000f007200061
:10bfd800808f5000e9ff3e006168800000c02000ab
:10bfe800008040001e4878000100e8006068880072
:10bff80061688000f00720000080600060688800a9
:10c00800806880000000e80080688800dbff370057
:10c018008560a9000080fa004f00be0000400600bd
:10c028000400fa00008fbe001e00be004309dd00b8
:10c03800cd01de00830171004301dd0000a0250071
:10c048002126200002024000838248001e00be0014
:10c058004409dd00cc01de00830171004401dd00ec
:10c068000400be0096d807000000e9000080fa002e
:10c07800000006000400fa00008fbe0021e2a900bb
:10c088009560a9009580a9008560a9008580a90010
:10c098000000eb0020688800206880001068880095
:10c0a80010688000006888000000eb008068880045
:10c0b8008068800070688800706880006068880008
:10c0c8002002a900012220009140780090cfb300ff
:10c0d80000c0600020e2b70020a2a9002082a900c9
:10c0e8002062a9001e00be00cdff07004011880095
:10c0f80023a2a90023e2a900910a20009140780018
:10c10800f0c8b30000c0600001c2b3000140700075
:10c11800a9e0b700a10a20009140780080cfb300c1
:10c1280000c060000004a000aae0b7009580a90044
:10c138008560a9009560a80021e2a8002342a80014
:10c148000080fa00000006000400fa00008fbe001c
:10c1580031e2a90097c0a90097e0a90087c0a9000b
:10c1680087e0a9000000eb00506888005068800054
:10c178004068880040688000306888000000eb0054
:10c18800b0688800b0688000a0688800a068800057
:10c19800906888003002a9000123200091407800af
:10c1a80090cfb30000c0600030e2b70030a2a90011
:10c1b8003082a9003062a9001e00be0098ff070067
:10c1c800c011880033a2a90033e2a9006a20a800a0
:10c1d800de82a800310b20009140780080cfb300a8
:10c1e80000c060000014a000b3e0b700310b2000cd
:10c1f80091407800f0c8b30000c060000044a0007f
:10c20800b3e0b70097e0a90087c0a90097c0a800cd
:10c2180031e2a8003342a8000080fa0000000600be
:10c228000000fa00806880000080fa000000060024
:10c238000000fa00206880000080fa000000060074
:10c248000200fa000040eb00004f780021042000b3
:10c258009140780000ceb30000c0700042e0b70003
:10c26800806880000000e0000d00320071688000e6
:10c2780000c0200000804000104f78000100e80056
:10c288007068880071688000f007200000806000f6
:10c2980070688800806880000000e9008068880075
:10c2a80042c0bf007f40600042e0b7001e80fb0034
:10c2b8000080fa00000006000400fa001007980049
:10c2c8000040eb00004f78002104200091407800e6
:10c2d80000ceb30000c0700042e0b7008068800064
:10c2e8000000e00006003200716880001e00900027
:10c2f8008080500000c0200000804000104f78006f
:10c3080042c0bf007f40600042e0b7001e80fb00d3
:10c318000080fa00000006000400fa002047980098
:10c328000000eb00000f7800210420009140780005
:10c3380000ceb30000c0700042e0b70095c0bf0057
:10c34800704060000004e00007003a002e409000b2
:10c358000080fb00201188009580a80010002000b4
:10c36800000f78001400370021688000f01f2000bb
:10c37800808f500010003e0001688000008020007f
:10c38800008040002e419000024878000100e8003b
:10c398000068880001688000f01f200000806000ad
:10c3a80000688800206880000000e8002068880095
:10c3b80010002000000f780042c0bf007f406000de
:10c3c80042e0b7001e0078000080fa000000060076
:10c3d8000400fa00204798000000eb00000f7800e6
:10c3e800210420009140780000ceb30000c0700006
:10c3f80042e0b700710920009140780000c8b300fe
:10c4080000c060000004e00007003a002e409000e1
:10c418000080fb00a011880097e0a8001000200011
:10c42800000f78001400370051688000f01f2000ca
:10c43800808f500010003e003168800000a020006e
:10c44800008040002e419000024878000100e8007a
:10c458003068880031688000f01f2000008060008c
:10c4680030688800506880000000e8005068880044
:10c4780010002000000f780042c0bf007f4060001d
:10c4880042e0b7001e0078000080fa0000000600b5
:10c498000200fa00000f7800060037001e0078003e
:10c4a800104078009cff07000000e000fbff32000e
:10c4b8001e0fe8001e007800104078000004e0001d
:10c4c800f6ff3a000080fa00000006000200fa00b9
:10c4d800000f7800060037001e0078001040780032
:10c4e800bbff07000000e000fbff32001e0fe80062
:10c4f8001e007800104078000004e000f6ff3a00c3
:10c508000080fa00000006000200fa00000f780020
:10c518000421a9000441a90041102000914078009d
:10c52800f0ccb30000c0600004e1b70004c1a9006a
:10c5380005a1a9001e0078006102b80084007800f7
:10c5480000a02500000bb8002026200000a0b9009c
:10c55800070178000001410000a0250000a8b900eb
:10c568000001410082037800823e20000300200081
:10c578000600be0052d707000000e9001008880036
:10c588000000eb0000088800510a20009140780064
:10c59800f0c8b30000c0600001c3b30001407000e0
:10c5a800a5e0b7008460a9009460a80005e1a80090
:10c5b8000080fa0000000600809fbe000000fa001c
:10c5c800207280000000e90020728800207280003c
:10c5d8000000e0000a003a00803e20002072880037
:10c5e8001000200030728800e0688000e10f5000e1
:10c5f80003003a00c06d80000000e800c06d8800ac
:10c60800707280008172800061004000e080480004
:10c6180070728800817288008460a9000080fa0026
:10c628004f00be00004006000600fa0020079800f0
:10c638002e0090006101b800707280008172800045
:10c64800001f410001974900010037000060fe000b
:10c658007072800081728000be0f1000ae8f1800cb
:10c66800faff3a000080fa00000006000000fa0015
:10c678001021a9000111200091407800f0ccb300ee
:10c6880000c0600010e1b70010c1a90011a1a90005
:10c6980094e0a90084e0a9000000eb0030088800bd
:10c6a800f0e12400600888000080fa00000006001d
:10c6b800801f78000400fa00e0688000e10f500055
:10c6c80002003a000040eb00ffedb7008780a900a8
:10c6d8000080fa004f007800004006000600fa00cb
:10c6e800200798002e0090006101b80000a02500e6
:10c6f8002126200002d7070061005000e080580082
:10c70800008fbe001e21a9001e61a800e1112000b3
:10c7180091407800f0ccb30000c060001ee1b70083
:10c728001ec1a9001fa1a9001e007800d00888001a
:10c738001e00be004008de0001002000e00888005e
:10c748009e00780000832f0000804000a008880029
:10c7580000832f00f1ff2f003e014000ae8148000a
:10c768000200be004008de0001002000c00888006a
:10c77800210b20009140780080cfb30000c06000fa
:10c788000024a000b2e0b7009780a9008780a90024
:10c798002c21a9002c61a800c1122000914078002a
:10c7a800f0ccb30000c060002ce1b7002cc1a90098
:10c7b8002da1a9001e007800400988001e00be00b7
:10c7c8004008de0001002000500988000000eb004e
:10c7d800100988000000eb0030098800c10b200018
:10c7e8009140780080cfb30000c060000024a00012
:10c7f800bce0b7009a00a9008a00a9001fe1a800c0
:10c808002de1a80013e1a9001221a900211120009f
:10c8180091407800f0ccb30000c0600012e1b7008e
:10c8280012c1a90013a1a900b00d2000700888004a
:10c838000000eb00500888008500a9009500a900b9
:10c848009780a8000080fa00000006000000fa00a7
:10c858000000eb0040728800400620009fff0700a0
:10c868000080fa00000006000000fa000000eb005b
:10c87800407288009780a9009a00a9008780a900c3
:10c888008a00a9000080fa00000006000000fa00f3
:10c8980010002000407288008780a9008a00a90043
:10c8a8009780a8009a00a8000080fa0000000600ff
:10c8b8000400fa001007980040728000000f78000a
:10c8c8001e00900085ff0700100020009e0f10003a
:10c8d80001003a00edff07000080fa0000000600a2
:10c8e8000200fa00000f78003c21a900c1132000c3
:10c8f8009140780000c3b30000c070003ce1b7006d
:10c908003cc1a9003da1a900f0c32900c0098800c5
:10c918001e00e00003003a000080eb00a009880038
:10c92800020037001e007800a0098800e10b2000f3
:10c938009140780080cfb30000c060003040b30061
:10c94800bee0b7008a80a9009a80a8000080fa009b
:10c9580000000600809fbe000000fa007072800090
:10c9680081728000e0718800f17188008a80a900d6
:10c978003de1a9000080fa004f00be00004006001b
:020000040000fa
:10c98800b80d000050000000020000000000000088
:10c998000001010001010100010101006400010022
:10c9a800000000000000a000400100000200b800e4
:10c9b8001ec53f000000000000010000cdcccc00e7
:10c9c8003d000000ae4781003f000000000000006d
:10c9d800000000000000000000010000010000004d
:10c9e80000010a00404000000000000000000000b4
:10c9f80000ff0100000000001c0d00009c0000006a
:10ca080000000000560e00000600000002000000b2
:10ca18000000000000000000080e000028000000d0
:10ca280000000000300e00001400000002000000aa
:10ca380000000000000000000000000000000000ee
:10ca480000000000000000000000000000080000d6
:10ca58001c05000000000000440e00001200000049
:10ca680002000000e80300000000000000000000d1
:10ca78000000000000000000000000005c0e000044
:10ca88000200000000000000be0f0000a00000002f
:10ca980002000000010000000000000000000a0081
:10caa800000000000000000000640000000000001a
:10cab80000000000e8030000000000000000100073
:10cac800270000000000000000a086000100000010
:10cad8000000000040420f0000000000000080003d
:10cae80096980000000000000000e100f505000035
:10caf8000000000000ca9a003b000000000000008f
:10cb0800e40b5400020000000000e800764817001b
:10cb1800000000000010a500d4e80000000000009c
:10cb2800a0724e0018090000000040007a10f300bf
:10cb38005a0000000080c600a47e8d00030000009b
:10cb480000c16f00f2862300000000008a5d7800b3
:10cb58004563010000006400a7b3b600e00d0000c3
:10cb680000e889000423c7008a0000005e10000066
:10cb78002a00000002000000286e75006c6c290075
:10cb8800003031003233340035363700383941004f
:10cb9800424344004546000030313200333435000a
:10cba800363738003961620063646500660000004a
:10cbb8005e0e00006001000002000000000000009e
:10cbc80000000000f03f00000000a0009999b900a3
:10cbd8003f0000000040e1007a843f0000000000b0
:10cbe800e04d6200503f00000000e000e2361a000d
:10cbf8003f0000000080b500f8e43e00000000009f
:10cc0800a0f7c600b03e00000000a000f2d77a00ee
:10cc18003e00000000e08e0079453e000000000064
:10cc2800e00b2e00113e00000000e000df7cdb007e
:10cc38003d0000000000a1009cc73b000000000070
:10cc4800004c4800b439000000000000206ca1002e
:10cc58003700000000000000000000000000000095
:10cc680000000000000000000000000000000000bc
:10cc780000000000000000000000000000000000ac
:10cc8800000000000000000000000000000000009c
:10cc9800000000000000000000000000000000008c
:10cca8000000000000000000000000000000f0008c
:10ccb8003f000000000000000024400000000000c9
:10ccc80000000000594000000000000000408f00f4
:10ccd800400000000000000088c340000000000081
:10cce80000006a00f84000000000000080842e0068
:10ccf800410000000000d000126341000000000065
:10cd08000084d700974100000000000065cdcd00e9
:10cd18004100000000205f00a00242000000000067
:10cd2800801daf001544000000004000593e290056
:10cd3800460000000000000000f07f000000000036
:10cd480000000000f07f0000000000000000f0007c
:10cd58007f0000000000000000f07f0000000000dd
:10cd680000000000f07f0000000000000000f0005c
:10cd78007f0000000000000000f07f0000000000bd
:10cd880000000000f07f0000000000000000f0003c
:10cd98007f0000008810000026000000020000004c
:10cda8008a10b00010000000b01009000000000058
:10cdb8000200ae0010000000ae10060002010000e4
:10cdc8000000000000000000000006000202000051
:10cdd80000000000ae100000060000000000000087
:10cde800b410000002000000020000000100000072
:04cdf8000000000037
:020000040000fa
:10cdfc000000fa008540a9009540a9004382a900d3
:10ce0c004362a9004342a9002124200091407800ec
:10ce1c00c0cfb30000c0600042e2b70042c2bf0006
:10ce2c00c041b30042e2b7004322a9004302a8006c
:10ce3c0042c2a90042a2a80041e2a8008540a90074
:10ce4c009540a9000080fa00000006000400fa00da
:10ce5c001007980040128000000f78008540a90050
:10ce6c000000000000000000000000001e00900008
:10ce7c004012880085c0bf00644060000004e000e0
:10ce8c00fcff320000000000000000000000000069
:10ce9c000080fa00000006000400fa002047980009
:10ceac0040128000004f78008540a900000000006f
:10cebc0000000000000000002e4090000080fb00ed
:10cecc004012880085c0bf00644060000004e00090
:10cedc00fcff320000000000000000000000000019
:10ceec000080fa00000006000000fa00c0ff0700f6
:10cefc007007a9002be3a8002a43a8002a23a80046
:10cf0c00e8c2a900e4c2a900800c200001002000a6
:10cf1c0040f00700e8c2a800e4c2a900007d200090
:10cf2c00010020003bf00700000320002000070058
:10cf3c00800c20000100200036f0070000032000c8
:10cf4c001b000700000320001900070090032000bd
:10cf5c0017000700400120001500070060052000a5
:10cf6c0013000700d0062000110007000007200066
:10cf7c000f000700c00020000d000700600020001b
:10cf8c000b0007001000200009000700803e200065
:10cf9c00010020001ff00700803e2000010020004f
:10cfac001cf00700c5e707000080fa00000006002f
:10cfbc000200fa00000f7800d042a900cc42a90070
:10cfcc00d022a900cc22a9001e007800b2ff0700d5
:10cfdc00d042a800cc42a9000080fa000000060054
:10cfec000200fa00000f7800d042a900cc42a90040
:10cffc00d022a800cc22a9001e007800a6ff0700b2
:10d00c00d042a800cc42a9000080fa000000060023
:10d01c000400fa001007980000c8b300004f780015
:10d02c000d0037001e80fb00e1ff070000c4290043
:10d03c0001002000f7ef07001e0090001040780060
:10d04c000000fb00e6ff07001e0090000000e80057
:10d05c00100798001e4fe8001e009000104078004a
:10d06c000004e000efff3a000080fa000000060028
:10d07c000400fa001007980000ccb300004f7800b1
:10d08c000d0037001e80fb00c9ff070000c42900fb
:10d09c0001002000dfef07001e0090001040780018
:10d0ac000000fb00ceff07001e0090000000e8000f
:10d0bc00100798001e4fe8001e00900010407800ea
:10d0cc000004e000efff3a000080fa0000000600c8
:10d0dc000000fa00313a800000e02f000080600070
:10d0ec00e104200001007000303a880041742000f7
:10d0fc009140780000ceb30000c0600044e7b70058
:10d10c0044c7bf00f043b20044e7b70043c7bf00b9
:10d11c00e740600043c7bf000080fb004400de0016
:10d12c006740600080cf5000f8ff3a000080fa00a2
:10d13c00000006004600fa00881f78000040eb0053
:10d14c0050479800e2ff070042c0bf007f406000dc
:10d15c0042e0b70000202c0011002000008fbe0020
:10d16c001e00be00c2fb07001e00be00f5fb070040
:10d17c00b5fd0700c522a900c122a8000000eb00e4
:10d18c0040708800e822a800e422a900e802a90067
:10d19c00e402a9000000eb009016880000f22b00be
:10d1ac00210020009bef070000f22b002100200043
:10d1bc0098ef070000f22b002100200095ef0700ec
:10d1cc0000f22b002100200092ef070000f22b0050
:10d1dc00210020008fef070000f22b00210020001f
:10d1ec008cef070000f22b002100200089ef0700d4
:10d1fc0000f22b002100200086ef070000f22b002c
:10d20c002100200083ef070000f22b0021002000fa
:10d21c0080ef070000f22b00210020007def0700bb
:10d22c0000f22b00210020007aef070000f22b0007
:10d23c002100200077ef07007dfa07001000200086
:10d24c00b0fc0700caee070001c2b30010c0b30067
:10d25c00dbf7070001c2b30020c0b300d8f707000a
:10d26c00110020008000200067f90700000000007a
:10d27c000000000000000000000000008000eb0037
:10d28c008000200060f9070012f8070016ff070065
:10d29c001c00370048708000e8fb070080407800d5
:10d2ac0010e120000000440001487800417080002b
:10d2bc0010e120000080400010407800ea4f500040
:10d2cc0004003200407080000000e80040708800cc
:10d2dc000c003700407080008000e80010e1200056
:10d2ec00808040000040eb008048780010e1200076
:10d2fc0066fc070011cebf003ff007000000eb00fa
:10d30c0040708800c5fb07000000e000e1ff3a0018
:10d31c0076ee070011f60700ddf5070054e807006c
:10d32c0042eb0700c9e7070028e80700f5ff3700c4
:020000040000fa
:08d33c000040da000000fe00d1
:00000001FF
